:020000040000FA
:1000000002EF00F00F01EB0E926E1F0E936E000ECA
:10001000946E000E956E0F0E966E030E386F000EE6
:10002000396F000E3A6F000E3B6F000E3C6F010EF1
:10003000C26E040EC16EB20EC06E700ED36E400E54
:100040009B6E806A816A826A836A846A896A8A6A24
:100050008B6A8C6A8D6A00018C8C006A016A026A64
:10006000036A046A056A066A076A086A096A0A6A0C
:100070000B6A0C6A0D6A0E6A0F6A106A116A126ABC
:10008000136A146A156A166A176A186A196A1A6A6C
:100090001B6A1C6A1D6A1E6A1F6A206A216A226A1C
:1000A000236A246A256A266A276A286A296A2A6ACC
:1000B0002B6A2C6A2D6A2E6A2F6A306A316A326A7C
:1000C000366A376A386A396A3A6A3B6A3C6A3D6A14
:1000D0003E6A3F6A406A416A426A436A446A456AC4
:1000E000466A476A486A496A4A6A4B6A4C6A4D6A74
:1000F0004E6A4F6A506A516A526A536A546A556A24
:10010000566A576A586A596A5A6A5B6A5C6A5D6AD3
:100110005E6A5F6A606B8C868088128C000EAA6EA5
:10012000000EA96EA69EA69CA68000000000A85006
:10013000486E000EAA6E010EA96EA69EA69CA68011
:1001400000000000A850496E000EAA6E020EA96EB3
:10015000A69EA69CA68000000000A8504A6E4A8079
:10016000000EAA6E030EA96EA69EA69CA680000095
:100170000000A8504B6E000EAA6E040EA96EA69E3B
:10018000A69CA68000000000A8504C6E000EAA6E2F
:10019000050EA96EA69EA69CA68000000000A85091
:1001A0004D6E000EAA6E060EA96EA69EA69CA68097
:1001B00000000000A850516E000EAA6E070EA96E36
:1001C000A69EA69CA68000000000A850376E000ED8
:1001D000AA6E080EA96EA69EA69CA680000000002E
:1001E000A850416E5150526E3750386E4150426E99
:1001F000A6EC27F0B1EC24F0C00E8B6E8C928C90A4
:100200000000000000000000000000008C840000DE
:1002100000000000000000000000000000000000DE
:1002200000000000000000000000000000000000CE
:1002300000000000000000000000000000008C949E
:1002400000000000000000000000000000000000AE
:10025000000000000000000000000000000000009E
:10026000000032EC25F03F0E8B6E8C928C900000DB
:10027000000000000000000000008C84000000006E
:10028000000000000000000000000000000000006E
:10029000000000000000000000000000000000005E
:1002A0000000000000000000000000008C9400002E
:1002B000000000000000000000000000000000003E
:1002C000000000000000000000000000000000002E
:1002D0001BEC26F08C8EB4EC24F0EBEC27F0C46A17
:1002E000C36A4A90120E476E4A50456E38EC26F0AB
:1002F000E7EC2CF0160E476E6EEC26F04E6E170EE5
:10030000476E6EEC26F04F6E6DEC2AF089EC2BF008
:1003100084B030EF02F00C0E3E5CD8B493EF01F0E5
:100320003E2A32EF02F03E6A11B832EF02F0118835
:10033000000E145CD8B4B3EF01F0010E145CD8B415
:10034000CEEF01F0020E145CD8B4D3EF01F0030E2F
:10035000145CD8B4EFEF01F0040E145CD8B404EFD1
:1003600002F01AEF02F04CBA32EF02F04CA2BDEFED
:1003700001F04C924C80C6EF01F04CA0C4EF01F0AC
:100380004C924C90C6EF01F04C824C90140E476E8C
:100390004C50456E38EC26F032EF02F0146A1BEC3C
:1003A00026F032EF02F012B0E2EF01F0196A12A269
:1003B0001A6A12A41B6A12A61C6A146A1BEC26F0A5
:1003C00032EF02F01FBAECEF01F01D6A196A1290C9
:1003D0001BEC26F032EF02F01F9A32EF02F012B25D
:1003E000FEEF01F01A6A12A0196A12A41B6A12A683
:1003F0001C6A146A1BEC26F032EF02F05150526E68
:100400001F98129232EF02F012B613EF02F01C6A3C
:1004100012A0196A12A21A6A12A41B6A146A1BECAF
:1004200026F032EF02F03750386E4150426E12968D
:1004300032EF02F012B429EF02F01B6A12A0196A1F
:1004400012A21A6A12A61C6A146A1BEC26F032EF7A
:1004500002F01BEC26F01B6A12941F9E32EF02F092
:1004600011983E6A6DEC2AF084B2C2EF04F00C0ED3
:100470003F5CD8B43FEF02F03F2AC4EF04F03F6A7C
:1004800011B6C4EF04F01186000E145CD8B45FEF0F
:1004900002F0010E145CD8B474EF02F0020E145C8A
:1004A000D8B476EF02F0030E145CD8B4EBEF03F08F
:1004B000040E145CD8B438EF04F04DEF04F04CBADD
:1004C000C4EF04F04CB8C4EF04F04BA26BEF02F0A1
:1004D0004B926CEF02F04B82130E476E4B50456E01
:1004E00038EC26F0C4EF04F0C4EF04F012B0AFEF24
:1004F00002F012801BEC26F0000E195CD8B497EFC6
:1005000002F0010E195CD8B49BEF02F0020E195CE8
:10051000D8B49FEF02F0030E195CD8B4A3EF02F039
:10052000040E195CD8B4A7EF02F0ABEF02F048500C
:10053000536EC4EF04F04950536EC4EF04F04A50B8
:10054000536EC4EF04F04B50536EC4EF04F04C50A4
:10055000536EC4EF04F04D50536EC4EF04F0080E18
:100560001D5CD8A40CEF03F0000E195CD8B4CFEFDB
:1005700002F0010E195CD8B4D9EF02F0020E195C3A
:10058000D8B4E3EF02F0030E195CD8B4EDEF02F03B
:10059000040E195CD8B4F7EF02F001EF03F05350EA
:1005A000486E100E476E4850456E38EC26F009EF45
:1005B00003F05350496E110E476E4950456E38ECAA
:1005C00026F009EF03F053504A6E120E476E4A5060
:1005D000456E38EC26F009EF03F053504B6E130EC6
:1005E000476E4B50456E38EC26F009EF03F0535040
:1005F0004C6E140E476E4C50456E38EC26F009EFE9
:1006000003F053504D6E150E476E4D50456E38EC4D
:1006100026F01D6AC4EF04F01FAA7DEF03F0000E60
:100620001D5CD8B434EF03F0010E1D5CD8B43DEF6F
:1006300003F0020E1D5CD8B446EF03F0030E1D5C00
:10064000D8B44FEF03F0040E1D5CD8B458EF03F09C
:10065000050E1D5CD8B461EF03F0060E1D5CD8B426
:100660006AEF03F073EF03F01FAC3AEF03F053802F
:100670007AEF03F053907AEF03F01FAC43EF03F0EF
:1006800053827AEF03F053927AEF03F01FAC4CEFF2
:1006900003F053847AEF03F053947AEF03F01FAC26
:1006A00055EF03F053867AEF03F053967AEF03F099
:1006B0001FAC5EEF03F053887AEF03F053987AEFA4
:1006C00003F01FAC67EF03F0538A7AEF03F0539AFD
:1006D0007AEF03F01FAC70EF03F0538C7AEF03F066
:1006E000539C7AEF03F01FAC79EF03F0538E7AEF4F
:1006F00003F0539E1F9AC4EF04F0000E1D5CD8B4A3
:10070000A2EF03F0010E1D5CD8B4ABEF03F0020EB4
:100710001D5CD8B4B4EF03F0030E1D5CD8B4BDEF7C
:1007200003F0040E1D5CD8B4C6EF03F0050E1D5C8B
:10073000D8B4CFEF03F0060E1D5CD8B4D8EF03F0A9
:10074000E1EF03F053A0A8EF03F01F8CE8EF03F0F4
:100750001F9CE8EF03F053A2B1EF03F01F8CE8EF0A
:1007600003F01F9CE8EF03F053A4BAEF03F01F8CD3
:10077000E8EF03F01F9CE8EF03F053A6C3EF03F08C
:100780001F8CE8EF03F01F9CE8EF03F053A8CCEFB9
:1007900003F01F8CE8EF03F01F9CE8EF03F053AA6F
:1007A000D5EF03F01F8CE8EF03F01F9CE8EF03F098
:1007B00053ACDEEF03F01F8CE8EF03F01F9CE8EF73
:1007C00003F053AEE7EF03F01F8CE8EF03F01F9C3C
:1007D0001F8AC4EF04F012B2F1EF03F01282C4EFEB
:1007E00004F05250516E12921FB8F9EF03F0C4EFAB
:1007F00004F0FF0E486EFF0E496EA00E4A6E010E09
:100800004B6E020E4C6E000E4D6E100E476E485031
:10081000456E38EC26F0110E476E4950456E38ECA7
:1008200026F0120E476E4A50456E38EC26F0130E35
:10083000476E4B50456E38EC26F0140E476E4C5008
:10084000456E38EC26F0150E476E4D50456E38EC6F
:1008500026F0000E516E000E526E000E376E000E26
:10086000386E010E416E010E426E1F98C4EF04F007
:1008700012B63EEF04F01286C4EF04F03850376E23
:100880004250416E276A286A296A2A6A2B6A2C6AB2
:100890002D6A2E6A1296C4EF04F012B455EF04F0DC
:1008A00012841BEC26F0C4EF04F01FBE5FEF04F0CF
:1008B0001BEC26F01B6A12941F9EC4EF04F0000E7E
:1008C0001B5CD8A468EF04F0E5EC3BF0BBEF04F050
:1008D000010E1B5CD8A471EF04F0F8EC3BF0BBEF09
:1008E00004F0020E1B5CD8A47AEF04F00BEC3CF091
:1008F000BBEF04F0030E1B5CD8A483EF04F01FECE5
:100900003CF0BBEF04F0040E1B5CD8A48CEF04F0A9
:1009100032EC3CF0BBEF04F0050E1B5CD8A495EF65
:1009200004F045EC3CF0BBEF04F0060E1B5CD8A4D1
:100930009EEF04F058EC3CF0BBEF04F0070E1B5C9C
:10094000D8A4A9EF04F06BEC3CF07EEC3CF0BBEFDC
:1009500004F0E5EC3BF0F8EC3BF00BEC3CF01FEC6A
:100960003CF032EC3CF045EC3CF058EC3CF06BECED
:100970003CF07EEC3CF01B6A1BEC26F012941F9EB0
:10098000C4EF04F011963F6A6DEC2AF084B4EBEFEB
:1009900004F00C0E3B5CD8B4D1EF04F03B2AEDEF31
:1009A00004F03B6A11BAEDEF04F0118A4AA0E2EFBD
:1009B00004F04A90120E476E4A50456E38EC26F00D
:1009C000EDEF04F04A80120E476E4A50456E38EC47
:1009D00026F0EDEF04F0119A3B6A6DEC2AF080BA34
:1009E0000CEF05F0070E405CD8B4FAEF04F0402A93
:1009F0000EEF05F0406A11B00EEF05F0050E145C25
:100A0000D8B406EF05F0142A07EF05F0146A1BECC2
:100A100026F011800EEF05F01190406A000E145C74
:100A2000D8B42EEF05F0010E145CD8B456EF0DF0DB
:100A3000020E145CD8B42BEF0FF0030E145CD8B484
:100A4000ACEF16F0040E145CD8B4C8EF1BF0050E22
:100A5000145CD8B465EF20F078EF01F0E7EC2CF0EF
:100A6000ABEC24F0410EB7EC24F0B80EDFEC24F030
:100A7000700E07EC25F0100E07EC25F0100E07ECB9
:100A800025F0100E07EC25F0000E07EC25F0AAEC7F
:100A900038F0000E07EC25F0EAEC37F0000E07EC1A
:100AA00025F07AEC38F0000E07EC25F0FAEC34F083
:100AB000000E07EC25F05AEC35F0000E07EC25F09F
:100AC0007AEC35F0000E07EC25F00AEC35F02AEC54
:100AD0003BF0DAEC38F0000E07EC25F0EAEC38F0E9
:100AE000AEEC24F0400EB7EC24F0B80EDFEC24F0AE
:100AF000CAEC37F0000E07EC25F0EAEC38F0000EF7
:100B000007EC25F0FAEC38F0000E07EC25F0DAECF3
:100B100038F0000E07EC25F0082A270E085CD8B440
:100B200097EF05F0100E07EC25F08CEF05F0086A42
:100B3000700E07EC25F0ABEC24F0410EB7EC24F07E
:100B4000BC0EDFEC24F0700E07EC25F0100E07EC65
:100B500025F0100E07EC25F0100E07EC25F0000E26
:100B600007EC25F06AEC38F02AEC3BF0EAEC37F0C1
:100B7000000E07EC25F03AEC38F0000E07EC25F0FB
:100B8000082A230E085CD8B4CBEF05F0100E07EC52
:100B900025F0C0EF05F0086A700E07EC25F0AEEC0A
:100BA00024F0410EB7EC24F0BC0EDFEC24F0700E04
:100BB00007EC25F0100E07EC25F0100E07EC25F0E1
:100BC000100E07EC25F0000E07EC25F0CAEC38F00B
:100BD0002AEC3BF0EAEC37F0000E07EC25F03AEC9B
:100BE00038F0000E07EC25F0082A230E085CD8B474
:100BF000FFEF05F0100E07EC25F0F4EF05F0086AA2
:100C0000700E07EC25F0ABEC24F0410EB7EC24F0AD
:100C1000BD0EDFEC24F0CAEC37F0000E07EC25F037
:100C20004EEC3BF0000E07EC25F0000E07EC25F033
:100C30004850506E4CBA28EF06F04CB828EF06F03A
:100C40004AAE28EF06F00F0E505CD8B04CEF06F01D
:100C50002AEC3BF0000E07EC25F0000E07EC25F027
:100C60006EEC3BF0000E07EC25F06EEC3BF0000E56
:100C700007EC25F06EEC3BF0000E07EC25F0400E83
:100C800007EC25F0000E07EC25F06EEC3BF0000EB3
:100C900007EC25F081EF06F05042509EFF0E485CB5
:100CA000D8B45DEF06F06EEC3BF0000E07EC25F0DB
:100CB000000E07EC25F065EF06F02AEC3BF0000E85
:100CC00007EC25F0000E07EC25F0501E509E50500A
:100CD00018EC2CF064EC2CF0400E07EC25F0000E24
:100CE00007EC25F048B07CEF06F03AEC35F0000E4A
:100CF00007EC25F081EF06F0EAEC34F0000E07EC8B
:100D000025F0000E07EC25F05AEC39F0000E07EC48
:100D100025F0DAEC37F0000E07EC25F0E7EC2CF0CC
:100D2000AEEC24F0420EB7EC24F0BD0EDFEC24F064
:100D3000CAEC37F0000E07EC25F04EEC3BF0000E4D
:100D400007EC25F04950506E4CBAB2EF06F04CB8A3
:100D5000B2EF06F04AAEB2EF06F00F0E505CD8B01C
:100D6000D6EF06F02AEC3BF0000E07EC25F0000E63
:100D700007EC25F06EEC3BF0000E07EC25F06EEC76
:100D80003BF0000E07EC25F06EEC3BF0000E07EC9C
:100D900025F0400E07EC25F0000E07EC25F06EEC78
:100DA0003BF0000E07EC25F00BEF07F05042509E91
:100DB000FF0E495CD8B4E7EF06F06EEC3BF0000E96
:100DC00007EC25F0000E07EC25F0EFEF06F02AEC1B
:100DD0003BF0000E07EC25F0000E07EC25F0501E4E
:100DE000509E505018EC2CF064EC2CF0400E07ECA8
:100DF00025F0000E07EC25F049B006EF07F03AECBD
:100E000035F0000E07EC25F00BEF07F0EAEC34F0BC
:100E1000000E07EC25F0000E07EC25F05AEC39F037
:100E2000000E07EC25F0DAEC37F0000E07EC25F0A9
:100E3000ABEC24F0400EB7EC24F0B90EDFEC24F05C
:100E40004CAA37EF07F0FF0E07EC25F0AAEC39F0BB
:100E5000FF0E07EC25F09AEC3AF0FF0E07EC25F0B8
:100E6000AAEC39F0FF0E07EC25F049EF07F0FF0E72
:100E700007EC25F06AEC3AF0FF0E07EC25F09AEC4F
:100E800039F0FF0E07EC25F03AEC3AF0FF0E07ECD4
:100E900025F0E7EC2CF0ABEC24F0550EB7EC24F089
:100EA000B90EDFEC24F04CBA90EF08F04AACD0EF6A
:100EB00007F04AAA61EF07F04CB890EF08F090EF06
:100EC00008F04AA882EF07F04CB890EF08F0FF0E48
:100ED00007EC25F0AAEC35F0FF0E07EC25F0CAEC84
:100EE00035F0FF0E07EC25F08AEC39F0FF0E07EC29
:100EF00025F0FAEC39F0FF0E07EC25F0AAEC3AF0F9
:100F00009BEF07F0FF0E07EC25F09AEC35F0FF0E93
:100F100007EC25F0EAEC35F0FF0E07EC25F08AEC43
:100F200039F0FF0E07EC25F0FAEC39F0FF0E07EC74
:100F300025F0AAEC3AF03AEC3BF0FAEC39F0FF0E6F
:100F400007EC25F0FF0E07EC25F0BD0E07EC25F0B1
:100F5000AEEC24F0400EB7EC24F0B90EDFEC24F038
:100F6000810E07EC25F0BD0E07EC25F0FF0E07EC17
:100F700025F0FF0E07EC25F09AEC3AF0FF0E07EC97
:100F800025F02AEC3BF0000E07EC25F0000E07ECF4
:100F900025F02AEC3BF0000E07EC25F0CFEF08F02F
:100FA0004AAA27EF08F04CA8D9EF07F04AB890EF0B
:100FB00008F0FF0E07EC25F0AAEC35F0FF0E07EC69
:100FC00025F0CAEC35F0FF0E07EC25F08AEC39F07D
:100FD000FF0E07EC25F0FAEC39F0FF0E07EC25F0D8
:100FE000AAEC3AF04AA85EEF08F03AEC3BF02AECA3
:100FF0003AF0FF0E07EC25F0EF0E07EC25F0EF0EB0
:1010000007EC25F0AEEC24F0400EB7EC24F0B90E5E
:10101000DFEC24F0EF0E07EC25F0EF0E07EC25F0E7
:10102000EF0E07EC25F0FF0E07EC25F00AEC3AF086
:10103000FF0E07EC25F09AEC3AF0FF0E07EC25F0D6
:10104000AAEC3AF0FF0E07EC25F0CFEF08F04AA823
:1010500045EF08F0FF0E07EC25F0AAEC35F0FF0E87
:1010600007EC25F08AEC35F0FF0E07EC25F08AEC52
:1010700039F0FF0E07EC25F0FAEC39F0FF0E07EC23
:1010800025F0AAEC3AF05EEF08F0FF0E07EC25F031
:101090009AEC35F0FF0E07EC25F0EAEC35F0FF0E88
:1010A00007EC25F08AEC39F0FF0E07EC25F0FAEC9E
:1010B00039F0FF0E07EC25F0AAEC3AF03AEC3BF0E1
:1010C0008AEC3AF0FF0E07EC25F0EF0E07EC25F066
:1010D000EF0E07EC25F0AEEC24F0400EB7EC24F058
:1010E000B90EDFEC24F0EF0E07EC25F0EF0E07EC65
:1010F00025F0EF0E07EC25F0FF0E07EC25F00AECCB
:101100003AF0FF0E07EC25F09AEC3AF0FF0E07ECF0
:1011100025F0AAEC3AF0FF0E07EC25F0CFEF08F02F
:10112000000E07EC25F02AEC3BF0000E07EC25F052
:101130002AEC3BF0000E07EC25F02AEC3BF0000E09
:1011400007EC25F02AEC3BF0000E07EC25F02AEC2A
:101150003BF0000E07EC25F02AEC3BF0000E07EC0C
:1011600025F02AEC3BF0000E07EC25F0AEEC24F065
:10117000400EB7EC24F0B90EDFEC24F02AEC3BF083
:10118000000E07EC25F02AEC3BF02AEC3BF0000EB9
:1011900007EC25F02AEC3BF0000E07EC25F036ECCE
:1011A0002FF0E7EC2CF0AEEC24F0580EB7EC24F066
:1011B000B90EDFEC24F04CBA1FEF09F04CB81FEF6A
:1011C00009F04AAE1FEF09F0FF0E07EC25F07AECAC
:1011D00039F0FF0E07EC25F0AAEC3AF0FF0E07EC11
:1011E00025F0AAEC3AF03AEC3BF051B204EF09F0EA
:1011F0002AEC3AF0FF0E07EC25F08AEC3AF0FF0EED
:1012000007EC25F03AEF09F051B413EF09F02AEC9E
:101210003AF0FF0E07EC25F03AEC3BF0FF0E07EC3E
:1012200025F03AEF09F03AEC3BF0FF0E07EC25F021
:101230008AEC3AF0FF0E07EC25F03AEF09F0000EC9
:1012400007EC25F02AEC3BF0000E07EC25F02AEC29
:101250003BF0000E07EC25F02AEC3BF02AEC3BF0CB
:101260002AEC3BF0000E07EC25F02AEC3BF0000ED8
:1012700007EC25F0ABEC24F0400EB7EC24F0BA0EEE
:10128000DFEC24F04CBA87EF09F04CB887EF09F097
:101290004BA269EF09F0FF0E07EC25F09AEC3AF04B
:1012A000FF0E07EC25F02AEC3AF0FF0E07EC25F0D4
:1012B0005AEC3AF0FF0E07EC25F0DAEC3AF0FF0EAC
:1012C00007EC25F02AEC3BF0000E07EC25F0A3EF2D
:1012D00009F0FF0E07EC25F09AEC3AF0FF0E07EC50
:1012E00025F0EAEC39F0FF0E07EC25F07AEC39F046
:1012F000FF0E07EC25F08AEC3AF0FF0E07EC25F024
:101300006AEC3AF0FF0E07EC25F0A3EF09F0000EAF
:1013100007EC25F02AEC3BF0000E07EC25F02AEC58
:101320003BF0000E07EC25F02AEC3BF0000E07EC3A
:1013300025F02AEC3BF0000E07EC25F02AEC3BF000
:10134000000E07EC25F0ABEC24F0610EB7EC24F0B6
:10135000BA0EDFEC24F04CA232EF0AF04CA0F0EF12
:1013600009F04CBAD2EF09F0000E07EC25F02AEC98
:101370003BF0000E07EC25F02AEC3BF0000E07ECEA
:1013800025F02AEC3BF0000E07EC25F02AEC3BF0B0
:10139000000E07EC25F02AEC3BF0000E07EC25F0E0
:1013A000F3EF0AF0FF0E07EC25F08AEC39F0FF0EA0
:1013B00007EC25F09AEC39F0FF0E07EC25F01AEC5B
:1013C0003AF0FF0E07EC25F09EEC3BF0FF0E07EC29
:1013D00025F0CAEC35F0000E07EC25F0F3EF0AF02B
:1013E0004CBAB4EF09F04CB814EF0AF0FF0E07EC5A
:1013F00025F09AEC35F0FF0E07EC25F0AAEC35F05D
:10140000FF0E07EC25F00AEC36F0FF0E07EC25F096
:10141000CAEC39F0FF0E07EC25F09AEC3AF0FF0E1B
:1014200007EC25F0F3EF0AF0000E07EC25F02AECAC
:101430003BF0000E07EC25F02AEC3BF0000E07EC29
:1014400025F09AEC35F0FF0E07EC25F0EAEC35F0CC
:10145000FF0E07EC25F0EAEC3AF0FF0E07EC25F062
:10146000F3EF0AF04CA095EF0AF04CBA59EF0AF0EE
:101470004CB877EF0AF02AEC3BF0000E07EC25F0B1
:10148000FF0E07EC25F0BAEC35F0FF0E07EC25F067
:10149000AAEC35F0FF0E07EC25F0CAEC39F0FF0E90
:1014A00007EC25F09AEC3AF0FF0E07EC25F0F3EF8D
:1014B0000AF0FF0E07EC25F08AEC39F0FF0E07EC7E
:1014C00025F09AEC39F0FF0E07EC25F01AEC3AF013
:1014D000FF0E07EC25F09EEC3BF0FF0E07EC25F02D
:1014E000AAEC35F0000E07EC25F0F3EF0AF0000E41
:1014F00007EC25F02AEC3BF0000E07EC25F02AEC77
:101500003BF0000E07EC25F02AEC3BF0FF0E07EC59
:1015100025F0CAEC35F0FF0E07EC25F0EAEC3AF0C6
:10152000FF0E07EC25F0F3EF0AF04CBAB9EF0AF022
:101530004CB8D7EF0AF02AEC3BF0000E07EC25F090
:10154000FF0E07EC25F0EAEC35F0FF0E07EC25F076
:10155000CAEC35F0FF0E07EC25F0CAEC39F0FF0EAF
:1015600007EC25F09AEC3AF0FF0E07EC25F0F3EFCC
:101570000AF0FF0E07EC25F08AEC39F0FF0E07ECBD
:1015800025F09AEC39F0FF0E07EC25F01AEC3AF052
:10159000FF0E07EC25F02AEC3BF0000E07EC25F0DF
:1015A0002AEC3BF0000E07EC25F0F3EF0AF0000EFA
:1015B00007EC25F02AEC3BF0000E07EC25F02AECB6
:1015C0003BF0000E07EC25F02AEC3BF0FF0E07EC99
:1015D00025F00AEC36F0FF0E07EC25F0EAEC3AF0C5
:1015E000FF0E07EC25F0E7EC2CF0AEEC24F05D0EDE
:1015F000B7EC24F0BA0EDFEC24F04AA019EF0BF0A0
:10160000FF0E07EC25F03AEC3AF0FF0E07EC25F060
:10161000BAEC3AF0FF0E07EC25F0AAEC3AF0FF0E18
:1016200007EC25F0BAEC39F0FF0E07EC25F030EFAF
:101630000BF0000E07EC25F02AEC3BF0000E07EC57
:1016400025F02AEC3BF0000E07EC25F02AEC3BF0ED
:10165000000E07EC25F02AEC3BF0000E07EC25F01D
:10166000AEEC24F0420EB7EC24F0BA0EDFEC24F01E
:101670004EA257EF0BF04EA057EF0BF0FF0E07EC0A
:1016800025F00AEC3BF0FF0E07EC25F0BAEC39F040
:10169000FF0E07EC25F08AEC3AF0FF0E07EC25F080
:1016A0005AEC3AF0FF0E07EC25F06EEF0BF0000E4F
:1016B00007EC25F02AEC3BF0000E07EC25F02AECB5
:1016C0003BF0000E07EC25F02AEC3BF0000E07EC97
:1016D00025F02AEC3BF0000E07EC25F0ABEC24F0F3
:1016E000400EB7EC24F0BB0EDFEC24F04CB8D8EF82
:1016F0000BF0FF0E07EC25F0AAEC39F0FF0E07EC1B
:1017000025F0CAEC39F03AEC3BF04CB6A8EF0BF000
:101710009AEC3AF0FF0E07EC25F0AAEC3AF0FF0E37
:1017200007EC25F0BAEC39F0FF0E07EC25F08AEC57
:101730003AF0FF0E07EC25F0BAEC39F0FF0E07EC9B
:1017400025F05AEC3AF0FF0E07EC25F025EF0CF0EF
:101750003AEC3AF0FF0E07EC25F05AEC3AF0FF0EA7
:1017600007EC25F04AEC3AF0FF0E07EC25F05AECB6
:101770003AF03AEC3BF04CB4CBEF0BF02AEC3AF0F9
:10178000FF0E07EC25F0000E07EC25F0000E07EC2D
:1017900025F025EF0CF08AEC3AF0FF0E07EC25F06F
:1017A000000E07EC25F0000E07EC25F025EF0CF0FD
:1017B0002AEC3BF0000E07EC25F02AEC3BF02AEC7B
:1017C0003BF0FF0E07EC25F04BB407EF0CF03AECC2
:1017D0003AF0FF0E07EC25F05AEC3AF0FF0E07EC5A
:1017E00025F04AEC3AF0FF0E07EC25F05AEC3AF0FF
:1017F000FF0E07EC25F02AEC3BF02AEC3BF0000E44
:1018000007EC25F0000E07EC25F025EF0CF09AEC24
:101810003AF0FF0E07EC25F0AAEC3AF0FF0E07ECC9
:1018200025F0BAEC39F0FF0E07EC25F08AEC3AF01F
:10183000FF0E07EC25F0BAEC39F0FF0E07EC25F0AF
:101840005AEC3AF0FF0E07EC25F036EC2FF0E7ECFF
:101850002CF0ABEC24F0770EB7EC24F0BB0EDFECF1
:1018600024F04CBA99EF0CF04AB264EF0CF0000E81
:1018700007EC25F02AEC3BF0000E07EC25F0000EFB
:1018800007EC25F0000E07EC25F0AEEC24F0400E3E
:10189000B7EC24F0BB0EDFEC24F0000E07EC25F0D3
:1018A000000E07EC25F02AEC3BF0000E07EC25F0CB
:1018B0002AEC3BF0000E07EC25F02AEC3BF0000E82
:1018C00007EC25F0E2EF0CF04AB46CEF0CF04AB6EE
:1018D0006CEF0CF037EF0CF0FF0E07EC25F0AAECE4
:1018E00039F0FF0E07EC25F0FF0E07EC25F0FF0E98
:1018F00007EC25F0AEEC24F0400EB7EC24F0BB0E64
:10190000DFEC24F0FF0E07EC25F0FF0E07EC25F0CE
:10191000BAEC39F0FF0E07EC25F03AEC3AF0FF0E86
:1019200007EC25F06AEC3AF0FF0E07EC25F0E2EF49
:101930000CF0FF0E07EC25F0CAEC39F0FF0E07ECB7
:1019400025F0FF0E07EC25F0BD0E07EC25F0AEEC00
:1019500024F0400EB7EC24F0BB0EDFEC24F0810E37
:1019600007EC25F0BD0E07EC25F0FF0E07EC25F087
:10197000FF0E07EC25F08AEC3AF03AEC3BF04AB661
:10198000D3EF0CF04AB4CCEF0CF09AEC35F0FF0E2C
:1019900007EC25F0E2EF0CF0AAEC35F0FF0E07ECB7
:1019A00025F0E2EF0CF04AB4DDEF0CF0BAEC35F0C4
:1019B000FF0E07EC25F0E2EF0CF0CAEC35F0FF0E5D
:1019C00007EC25F0AEEC24F0560EB7EC24F0BB0E7D
:1019D000DFEC24F051B00FEF0DF0000E07EC25F016
:1019E0002AEC3BF0000E07EC25F02AEC3BF02AEC49
:1019F0003BF02AEC3BF0000E07EC25F02AEC3BF024
:101A0000000E07EC25F02AEC3BF0000E07EC25F069
:101A10002AEC3BF0000E07EC25F054EF0DF012BC61
:101A200034EF0DF0FF0E07EC25F0CAEC39F0FF0E95
:101A300007EC25F0FAEC3AF03AEC3BF02AEC3AF0FD
:101A4000FF0E07EC25F0FAEC39F0FF0E07EC25F05D
:101A50004AEC3AF0FF0E07EC25F01AEC3AF0FF0ED4
:101A600007EC25F054EF0DF0000E07EC25F01AEC12
:101A700038F0000E07EC25F03AEC39F02AEC3BF098
:101A80006AEC38F0000E07EC25F04AEC38F0000E56
:101A900007EC25F08AEC38F0000E07EC25F05AEC44
:101AA00038F0000E07EC25F078EF01F0ABEC24F0F5
:101AB000410EB7EC24F0B80EDFEC24F0700E07EC0A
:101AC00025F0100E07EC25F0100E07EC25F0100E97
:101AD00007EC25F0000E07EC25F0AAEC38F0000E1C
:101AE00007EC25F0EAEC37F0000E07EC25F07AEC75
:101AF00038F0000E07EC25F0FAEC34F0000E07EC9D
:101B000025F05AEC35F0000E07EC25F07AEC35F0B4
:101B1000000E07EC25F00AEC35F02AEC3BF0CAEC9D
:101B200038F0000E07EC25F00AEC38F0AEEC24F0AB
:101B3000400EB7EC24F0B80EDFEC24F02AEC38F0BD
:101B4000000E07EC25F04AEC38F0000E07EC25F00B
:101B5000DAEC38F0000E07EC25F0EAEC38F0000E75
:101B600007EC25F00AEC38F0000E07EC25F0CAEC83
:101B700038F0000E07EC25F0082A1B0E085CD8B4DC
:101B8000C7EF0DF0100E07EC25F0BCEF0DF0086A62
:101B9000700E07EC25F0ABEC24F0410EB7EC24F00E
:101BA000B90EDFEC24F0FF0E07EC25F07AEC39F0EB
:101BB000FF0E07EC25F0AAEC39F0FF0E07EC25F03C
:101BC000AAEC39F0FF0E07EC25F08AEC3AF0FF0E94
:101BD00007EC25F0BAEC39F0FF0E07EC25F09AEC93
:101BE0003AF0FF0E07EC25F09AEC3AF0FF0E07EC06
:101BF00025F0AEEC24F0410EB7EC24F0B90EDFEC8A
:101C000024F0FF0E07EC25F0AAEC39F0FF0E07ECEC
:101C100025F07AEC39F0FF0E07EC25F0AAEC3AF04B
:101C2000FF0E07EC25F07AEC39F0FF0E07EC25F0FB
:101C3000ABEC24F0410EB7EC24F0BA0EDFEC24F04C
:101C4000000E155CD8B427EF0EF0EDEF0EF0FAECB5
:101C500034F0000E07EC25F04AEC35F0000E07ECEE
:101C600025F0FAEC37F0000E07EC25F0AEEC24F08E
:101C7000410EB7EC24F0BA0EDFEC24F0485090ECA3
:101C80002CF0ABEC24F0410EB7EC24F0BB0EDFECF3
:101C900024F0FAEC34F0000E07EC25F05AEC35F0A5
:101CA000000E07EC25F0FAEC37F0000E07EC25F0FB
:101CB000AEEC24F0410EB7EC24F0BB0EDFEC24F0C8
:101CC000495090EC2CF0ABEC24F0410EB7EC24F032
:101CD000BC0EDFEC24F0FAEC34F0000E07EC25F03B
:101CE0006AEC35F0000E07EC25F0FAEC37F0000E48
:101CF00007EC25F0AEEC24F0410EB7EC24F0BC0E5E
:101D0000DFEC24F04A5090EC2CF0ABEC24F0410EC8
:101D1000B7EC24F0BD0EDFEC24F0FAEC34F0000E4A
:101D200007EC25F07AEC35F0000E07EC25F0FAEC24
:101D300037F0000E07EC25F0AEEC24F0410EB7ECC6
:101D400024F0BD0EDFEC24F04B5090EC2CF0ABEC0B
:101D500024F0410EB7EC24F0BE0EDFEC24F00AECC8
:101D600035F0000E07EC25F0EAEC34F0000E07EC3D
:101D700025F0FAEC37F0000E07EC25F0AEEC24F07D
:101D8000410EB7EC24F0BE0EDFEC24F04C5090EC8A
:101D90002CF0ABEC24F0410EB7EC24F0BF0EDFECDE
:101DA00024F00AEC35F0000E07EC25F0FAEC34F0E4
:101DB000000E07EC25F0FAEC37F0000E07EC25F0EA
:101DC000AEEC24F0410EB7EC24F0BF0EDFEC24F0B3
:101DD0004D5090EC2CF029EF0FF00AEC35F0000E8E
:101DE00007EC25F00AEC35F0000E07EC25F0FAECD4
:101DF00037F0000E07EC25F0AEEC24F0410EB7EC06
:101E000024F0BA0EDFEC24F04E5090EC2CF0ABEC4A
:101E100024F0410EB7EC24F0BB0EDFEC24F00AEC0A
:101E200035F0000E07EC25F01AEC35F0000E07EC4B
:101E300025F0FAEC37F0000E07EC25F0AEEC24F0BC
:101E4000410EB7EC24F0BB0EDFEC24F04F5090ECC9
:101E50002CF078EF01F0ABEC24F0410EB7EC24F05D
:101E6000B80EDFEC24F0700E07EC25F0100E07EC36
:101E700025F0100E07EC25F0100E07EC25F0000EF3
:101E800007EC25F0AAEC38F0000E07EC25F0EAECA0
:101E900037F0000E07EC25F07AEC38F0000E07EC76
:101EA00025F0FAEC34F0000E07EC25F05AEC35F092
:101EB000000E07EC25F07AEC35F0000E07EC25F06B
:101EC0000AEC35F02AEC3BF0DAEC38F0000E07ECC7
:101ED00025F00AEC38F0AEEC24F0400EB7EC24F01C
:101EE000B80EDFEC24F0EAEC38F0000E07EC25F039
:101EF000EAEC38F0000E07EC25F04AEC38F0000E62
:101F000007EC25F08AEC38F0000E07EC25F02AECFF
:101F100038F0000E07EC25F0082A210E085CD8B432
:101F200097EF0FF0100E07EC25F08CEF0FF0086A1A
:101F3000700E07EC25F012B025EF11F0ABEC24F099
:101F4000460EB7EC24F0B90EDFEC24F0DAEC38F0F2
:101F5000000E07EC25F00AEC38F0000E07EC25F037
:101F60006AEC38F0000E07EC25F00AEC38F0000EB1
:101F700007EC25F0EAEC37F0000E07EC25F0EAEC70
:101F800038F0000E07EC25F02AEC3BF0CAEC37F0F5
:101F9000000E07EC25F0FAEC37F0000E07EC25F008
:101FA000FAEC37F0AEEC24F0400EB7EC24F0B90EAA
:101FB000DFEC24F0000E07EC25F0CAEC38F0000E40
:101FC00007EC25F00AEC38F0000E07EC25F0DAEC0F
:101FD00038F0000E07EC25F0DAEC38F0000E07ECD4
:101FE00025F0ABEC24F04A0EB7EC24F0BB0EDFEC8E
:101FF00024F0000E195CD8B412EF10F0000E07ECBC
:1020000025F0FAEC34F0000E07EC25F04AEC35F040
:10201000000E07EC25F0FAEC37F0000E07EC25F087
:1020200024EF10F0FF0E07EC25F09AEC35F0FF0ED0
:1020300007EC25F0EAEC35F0FF0E07EC25F0AAECF2
:1020400039F0FF0E07EC25F0ABEC24F0670EB7EC8F
:1020500024F0BB0EDFEC24F0010E195CD8B445EF80
:1020600010F0000E07EC25F0FAEC34F0000E07EC4F
:1020700025F05AEC35F0000E07EC25F0FAEC37F0BD
:10208000000E07EC25F057EF10F0FF0E07EC25F0DF
:102090009AEC35F0FF0E07EC25F0FAEC35F0FF0E68
:1020A00007EC25F0AAEC39F0FF0E07EC25F0AEECBA
:1020B00024F0440EB7EC24F0BB0EDFEC24F0020E4B
:1020C000195CD8B478EF10F0000E07EC25F0FAECAC
:1020D00034F0000E07EC25F06AEC35F0000E07EC4A
:1020E00025F0FAEC37F0000E07EC25F08AEF10F03F
:1020F000FF0E07EC25F09AEC35F0FF0E07EC25F00B
:102100000AEC36F0FF0E07EC25F0AAEC39F0FF0ED2
:1021100007EC25F0AEEC24F0610EB7EC24F0BB0E1A
:10212000DFEC24F0030E195CD8B4ABEF10F0000E16
:1021300007EC25F0FAEC34F0000E07EC25F07AEC11
:1021400035F0000E07EC25F0FAEC37F0000E07EC46
:1021500025F0BDEF10F0FF0E07EC25F09AEC35F0FE
:10216000FF0E07EC25F01AEC36F0FF0E07EC25F019
:10217000AAEC39F0FF0E07EC25F0ABEC24F04A0E88
:10218000B7EC24F0BC0EDFEC24F0040E195CD8B4DC
:10219000DEEF10F0000E07EC25F00AEC35F0000E33
:1021A00007EC25F0EAEC34F0000E07EC25F0FAEC31
:1021B00037F0000E07EC25F0F0EF10F0FF0E07EC03
:1021C00025F0AAEC35F0FF0E07EC25F08AEC35F08F
:1021D000FF0E07EC25F0AAEC39F0FF0E07EC25F016
:1021E000ABEC24F0670EB7EC24F0BC0EDFEC24F06F
:1021F000050E195CD8B411EF11F0000E07EC25F0B4
:102200000AEC35F0000E07EC25F0FAEC34F0000E85
:1022100007EC25F0FAEC37F0000E07EC25F023EF81
:1022200011F0FF0E07EC25F0AAEC35F0FF0E07ECDD
:1022300025F09AEC35F0FF0E07EC25F0AAEC39F00A
:10224000FF0E07EC25F078EF01F0ABEC24F0460E22
:10225000B7EC24F0B90EDFEC24F0000E195CD8B412
:1022600048EF11F0010E195CD8B4E6EF11F0020E40
:10227000195CD8B486EF12F0030E195CD8B48FEF56
:1022800013F0040E195CD8B498EF14F0A1EF15F018
:10229000C2EC3BF0FAEC34F0000E07EC25F04AEC0F
:1022A00035F0000E07EC25F0AEEC24F0400EB7EC54
:1022B00024F0B90EDFEC24F0FAEC37F0ABEC24F0AC
:1022C000460EB7EC24F0BC0EDFEC24F0080E1D5CCB
:1022D000D8B4D8EF11F0FF0E07EC25F07AEC39F006
:1022E000FF0E07EC25F0AAEC3AF0FF0E07EC25F004
:1022F0002AEC3AF0FF0E07EC25F0000E1D5CD8B476
:10230000A2EF11F0010E1D5CD8B4A9EF11F0020E7E
:102310001D5CD8B4B0EF11F0030E1D5CD8B4B7EF5C
:1023200011F0040E1D5CD8B4BEEF11F0050E1D5C5B
:10233000D8B4C5EF11F0060E1D5CD8B4CCEF11F087
:10234000D3EF11F08AEC35F0FF0E07EC25F0E2EF49
:1023500011F09AEC35F0FF0E07EC25F0E2EF11F0EA
:10236000AAEC35F0FF0E07EC25F0E2EF11F0BAEC25
:1023700035F0FF0E07EC25F0E2EF11F0CAEC35F076
:10238000FF0E07EC25F0E2EF11F0DAEC35F0FF0E6E
:1023900007EC25F0E2EF11F0EAEC35F0FF0E07EC68
:1023A00025F0E2EF11F0FAEC35F0FF0E07EC25F026
:1023B0002AEC3BF02AEC3BF02AEC3BF02AEC3BF019
:1023C0002AEC3BF0D1EC33F03EEF16F0C2EC3BF0E0
:1023D000FAEC34F0000E07EC25F05AEC35F0000E64
:1023E00007EC25F0AEEC24F0400EB7EC24F0B90E6B
:1023F000DFEC24F0FAEC37F0ABEC24F0460EB7EC4F
:1024000024F0BC0EDFEC24F0080E1D5CD8B478EF8D
:1024100012F0FF0E07EC25F07AEC39F0FF0E07EC16
:1024200025F0AAEC3AF0FF0E07EC25F08AEC3AF022
:10243000FF0E07EC25F0000E1D5CD8B440EF12F043
:10244000010E1D5CD8B447EF12F0020E1D5CD8B42B
:102450004EEF12F0030E1D5CD8B455EF12F0040ECF
:102460001D5CD8B45CEF12F0050E1D5CD8B463EFB0
:1024700012F0060E1D5CD8B46AEF12F071EF12F084
:102480008AEC35F0FF0E07EC25F082EF12F09AECA3
:1024900035F0FF0E07EC25F082EF12F0AAEC35F0D4
:1024A000FF0E07EC25F082EF12F0BAEC35F0FF0ECC
:1024B00007EC25F082EF12F0CAEC35F0FF0E07ECC6
:1024C00025F082EF12F0DAEC35F0FF0E07EC25F084
:1024D00082EF12F0EAEC35F0FF0E07EC25F082EF08
:1024E00012F0FAEC35F0FF0E07EC25F082EF12F057
:1024F0002AEC3BF02AEC3BF02AEC3BF02AEC3BF0D8
:102500002AEC3BF0D1EC33F03EEF16F0C2EC3BF09E
:10251000FAEC34F0000E07EC25F06AEC35F0000E12
:1025200007EC25F0AEEC24F0400EB7EC24F0B90E29
:10253000DFEC24F0FAEC37F0ABEC24F0460EB7EC0D
:1025400024F0BC0EDFEC24F0080E1D5CD8B481EF43
:1025500013F0FF0E07EC25F0000E1D5CD8B4D1EF90
:1025600012F0010E1D5CD8B4E7EF12F0020E1D5CF4
:10257000D8B4FDEF12F0030E1D5CD8B413EF13F0C6
:10258000040E1D5CD8B429EF13F0050E1D5CD8B401
:102590003FEF13F0060E1D5CD8B455EF13F06BEF50
:1025A00013F03AEC3AF0FF0E07EC25F0BAEC3AF0F3
:1025B000FF0E07EC25F0AAEC3AF0FF0E07EC25F031
:1025C000BAEC39F0FF0E07EC25F08BEF13F0AAEC14
:1025D00039F0FF0E07EC25F03AEC3AF0FF0E07EC6D
:1025E00025F0BAEC39F0FF0E07EC25F02AEC3BF0B1
:1025F000000E07EC25F08BEF13F0AAEC39F0FF0E7C
:1026000007EC25F03AEC3AF0FF0E07EC25F0CAECA7
:1026100039F0FF0E07EC25F08AEC35F0FF0E07ECE1
:1026200025F08BEF13F0AAEC39F0FF0E07EC25F044
:102630003AEC3AF0FF0E07EC25F0CAEC39F0FF0E49
:1026400007EC25F09AEC35F0FF0E07EC25F08BEF48
:1026500013F0CAEC39F0FF0E07EC25F03AEC3AF033
:10266000FF0E07EC25F0AAEC3AF0FF0E07EC25F080
:102670008AEC35F0FF0E07EC25F08BEF13F0CAEC77
:1026800039F0FF0E07EC25F03AEC3AF0FF0E07ECBC
:1026900025F0AAEC3AF0FF0E07EC25F09AEC35F0A5
:1026A000FF0E07EC25F08BEF13F0CAEC39F0FF0EAC
:1026B00007EC25F03AEC3AF0FF0E07EC25F0AAEC17
:1026C0003AF0FF0E07EC25F0AAEC35F0FF0E07EC10
:1026D00025F08BEF13F07AEC39F0FF0E07EC25F0C4
:1026E000AAEC3AF0FF0E07EC25F02AEC3AF0FF0EC8
:1026F00007EC25F0AAEC39F0FF0E07EC25F08BEF84
:1027000013F02AEC3BF02AEC3BF02AEC3BF02AECED
:102710003BF02AEC3BF0D1EC33F03EEF16F0C2EC8C
:102720003BF0FAEC34F0000E07EC25F07AEC35F0D3
:10273000000E07EC25F0AEEC24F0400EB7EC24F0D0
:10274000B90EDFEC24F0FAEC37F0ABEC24F0460ED7
:10275000B7EC24F0BC0EDFEC24F0080E1D5CD8B4FE
:102760008AEF14F0FF0E07EC25F0000E1D5CD8B4C4
:10277000DAEF13F0010E1D5CD8B4F0EF13F0020E87
:102780001D5CD8B406EF14F0040E1D5CD8B41CEF29
:1027900014F0050E1D5CD8B432EF14F0060E1D5C6B
:1027A000D8B448EF14F0070E1D5CD8B45EEF14F0F7
:1027B00074EF14F0FAEC39F0FF0E07EC25F04AEC58
:1027C0003AF0FF0E07EC25F00AEC3BF0FF0E07ECA9
:1027D00025F0AAEC39F0FF0E07EC25F094EF14F089
:1027E000CAEC39F0FF0E07EC25F02AEC3AF0FF0EA8
:1027F00007EC25F0AAEC3AF0FF0E07EC25F02AECE6
:102800003BF0000E07EC25F094EF14F0AAEC39F041
:10281000FF0E07EC25F0CAEC39F0FF0E07EC25F0AF
:102820003AEC3AF0FF0E07EC25F09AEC3AF0FF0E86
:1028300007EC25F094EF14F05AEC3AF0FF0E07EC99
:1028400025F06AEC3AF0FF0E07EC25F0BAEC39F00F
:10285000FF0E07EC25F02AEC3BF0000E07EC25F00C
:1028600094EF14F07AEC39F0FF0E07EC25F0AAECA7
:102870003AF0FF0E07EC25F09AEC3AF0FF0E07EC69
:1028800025F08AEC35F0FF0E07EC25F094EF14F0FC
:102890007AEC39F0FF0E07EC25F0AAEC3AF0FF0EC7
:1028A00007EC25F09AEC3AF0FF0E07EC25F09AECD5
:1028B00035F0FF0E07EC25F094EF14F08AEC3AF0B7
:1028C000FF0E07EC25F0BAEC39F0FF0E07EC25F00F
:1028D000CAEC3AF0FF0E07EC25F02AEC3BF0000EB4
:1028E00007EC25F094EF14F08AEC3AF0FF0E07ECB9
:1028F00025F09AEC3AF0FF0E07EC25F0CAEC3AF01E
:10290000FF0E07EC25F02AEC3BF0000E07EC25F05B
:1029100094EF14F02AEC3BF02AEC3BF02AEC3BF06D
:102920002AEC3BF02AEC3BF0D1EC33F03EEF16F012
:10293000C2EC3BF00AEC35F0000E07EC25F0EAECB7
:1029400034F0000E07EC25F0AEEC24F0400EB7ECAE
:1029500024F0B90EDFEC24F0FAEC37F0ABEC24F005
:10296000460EB7EC24F0BC0EDFEC24F0080E1D5C24
:10297000D8B493EF15F0FF0E07EC25F0000E1D5CA8
:10298000D8B4E3EF14F0010E1D5CD8B4F9EF14F0E5
:10299000020E1D5CD8B40FEF15F0030E1D5CD8B409
:1029A00025EF15F0040E1D5CD8B43BEF15F0050EB5
:1029B0001D5CD8B451EF15F0060E1D5CD8B467EF5E
:1029C00015F07DEF15F05AEC3AF0FF0E07EC25F00C
:1029D0009AEC3AF0FF0E07EC25F08AEC35F0FF0E8A
:1029E00007EC25F02AEC3BF0000E07EC25F09DEFFC
:1029F00015F05AEC3AF0FF0E07EC25F09AEC3AF09D
:102A0000FF0E07EC25F09AEC35F0FF0E07EC25F0F1
:102A10002AEC3BF0000E07EC25F09DEF15F09AEC48
:102A200039F0FF0E07EC25F0EAEC39F0FF0E07EC69
:102A300025F09AEC3AF0FF0E07EC25F02AEC3AF07C
:102A4000FF0E07EC25F09DEF15F03AEC3AF0FF0E83
:102A500007EC25F05AEC3AF0FF0E07EC25F04AECB3
:102A60003AF0FF0E07EC25F05AEC3AF0FF0E07ECB7
:102A700025F09DEF15F0AAEC39F0FF0E07EC25F0DC
:102A8000CAEC39F0FF0E07EC25F0AAEC3AF0FF0E85
:102A900007EC25F0EAEC39F0FF0E07EC25F09DEF8E
:102AA00015F0AAEC39F0FF0E07EC25F09AEC3AF09D
:102AB000FF0E07EC25F0AAEC39F0FF0E07EC25F02D
:102AC0002AEC3BF0000E07EC25F09DEF15F09AEC98
:102AD0003AF0FF0E07EC25F08AEC3AF0FF0E07EC17
:102AE00025F09AEC3AF0FF0E07EC25F0AAEC3AF04C
:102AF000FF0E07EC25F09DEF15F08AEC3AF0FF0E83
:102B000007EC25F09AEC3AF0FF0E07EC25F0CAEC42
:102B10003AF0FF0E07EC25F02AEC3BF0000E07EC34
:102B200025F09DEF15F02AEC3BF02AEC3BF02AEC67
:102B30003BF02AEC3BF02AEC3BF0D1EC33F03EEFDB
:102B400016F0C2EC3BF00AEC35F0000E07EC25F075
:102B5000FAEC34F0000E07EC25F0AEEC24F0400E59
:102B6000B7EC24F0B90EDFEC24F0FAEC37F0ABEC64
:102B700024F0460EB7EC24F0BC0EDFEC24F0080E77
:102B80001D5CD8B430EF16F0FF0E07EC25F0000EF8
:102B90001D5CD8B4D8EF15F0010E1D5CD8B4EEEF73
:102BA00015F0020E1D5CD8B404EF16F01AEF16F003
:102BB0006AEC3AF0FF0E07EC25F09AEC39F0FF0EC4
:102BC00007EC25F03AEC3AF0FF0E07EC25F00AECA2
:102BD0003BF0FF0E07EC25F03AEF16F0AAEC39F0C7
:102BE000FF0E07EC25F00AEC3BF0FF0E07EC25F09A
:102BF0008AEC35F0FF0E07EC25F02AEC3BF0000ED6
:102C000007EC25F03AEF16F0AAEC39F0FF0E07ECCE
:102C100025F00AEC3BF0FF0E07EC25F09AEC35F0BE
:102C2000FF0E07EC25F02AEC3BF0000E07EC25F038
:102C30003AEF16F08AEC3AF0FF0E07EC25F09AEC2A
:102C40003AF0FF0E07EC25F0CAEC3AF0FF0E07EC65
:102C500025F02AEC3BF0000E07EC25F03AEF16F0D9
:102C60002AEC3BF02AEC3BF02AEC3BF02AEC3BF060
:102C70002AEC3BF0D1EC33F03EEF16F0ABEC24F055
:102C80004D0EB7EC24F0BE0EDFEC24F01FBA69EF56
:102C900016F0000E07EC25F02AEC3BF0000E07ECD6
:102CA00025F02AEC3BF02AEC3BF0000E07EC25F077
:102CB0002AEC3BF0000E07EC25F02AEC3BF0000E6E
:102CC00007EC25F02AEC3BF0000E07EC25F0AAEF0C
:102CD00016F01FAC8CEF16F0FF0E07EC25F09AEC07
:102CE00035F0FF0E07EC25F02AEC3BF09AEC38F0BB
:102CF000000E07EC25F0CAEC38F0000E07EC25F0CA
:102D00002AEC3BF0000E07EC25F0EAEC34F0000E64
:102D100007EC25F0AAEF16F0000E07EC25F0FAEC10
:102D200034F0000E07EC25F02AEC3BF09AEC38F07A
:102D3000000E07EC25F0CAEC38F0000E07EC25F089
:102D40002AEC3BF0FF0E07EC25F08AEC35F0FF0E85
:102D500007EC25F078EF01F0ABEC24F0410EB7EC76
:102D600024F0B80EDFEC24F0700E07EC25F0100E06
:102D700007EC25F0100E07EC25F0100E07EC25F0FF
:102D8000000E07EC25F09AEC38F0000E07EC25F069
:102D9000EAEC38F0000E07EC25F03AEC38F0000EC3
:102DA00007EC25F00AEC38F0000E07EC25F0CAEC31
:102DB00038F0000E07EC25F02AEC3BF0DAEC38F0A6
:102DC000000E07EC25F00AEC38F0000E07EC25F0B9
:102DD000EAEC38F0000E07EC25F0EAEC38F0AEEC47
:102DE00024F0400EB7EC24F0B80EDFEC24F0000E17
:102DF00007EC25F04AEC38F0000E07EC25F08AECE1
:102E000038F0000E07EC25F02AEC38F0000E07EC45
:102E100025F0082A2C0E085CD8B414EF17F0100E19
:102E200007EC25F009EF17F0086A700E07EC25F0A3
:102E3000ABEC24F0460EB7EC24F0BF0EDFEC24F030
:102E4000DAEC38F0000E07EC25F09AEC38F0000EC2
:102E500007EC25F01AEC38F0000E07EC25F0EAEC50
:102E600038F0000E07EC25F01AEC39F0000E07ECF4
:102E700025F0CAEC37F0000E07EC25F0CAEC38F06C
:102E8000000E07EC25F00AEC38F0000E07EC25F0F8
:102E90002AEC3BF00AEC39F0AEEC24F0400EB7EC33
:102EA00024F0BF0EDFEC24F0000E07EC25F00AEC56
:102EB00038F0000E07EC25F0CAEC38F0000E07ECF5
:102EC00025F0DAEC38F0000E07EC25F04AEC38F08B
:102ED000000E07EC25F09AEC38F0000E07EC25F018
:102EE0008AEC38F0000E07EC25F02AEC3BF0000EDF
:102EF00007EC25F0FAEC34F0000E07EC25F0000E9C
:102F000007EC25F0400E07EC25F0000E07EC25F04D
:102F1000EAEC34F0000E07EC25F0EAEC34F0000E99
:102F200007EC25F0ABEC24F0400EB7EC24F0B90E22
:102F3000DFEC24F012B2A2EF17F0000E1A5CD8B446
:102F40000AEF18F0000E07EC25F0CAEC37F0000E7F
:102F500007EC25F0EAEC38F0000E07EC25F0EAEC7F
:102F600038F02AEC3BF06AEC38F0000E07EC25F064
:102F7000000E07EC25F08EEC3BF0000E07EC25F080
:102F8000000E07EC25F0CAEC38F02AEC3BF0EAEC36
:102F900037F0000E07EC25F03AEC38F02AEC3BF065
:102FA0003C0E07EC25F0AEEC24F0400EB7EC24F01C
:102FB000B90EDFEC24F0420E07EC25F0420E07ECD0
:102FC00025F0420E07EC25F0240E07EC25F0000E4C
:102FD00007EC25F09AEC38F0000E07EC25F08AECAF
:102FE00038F0000E07EC25F0EAEC38F0000E07ECA4
:102FF00025F0CAEC38F0000E07EC25F09AEC38F01A
:10300000000E07EC25F06AEC38F0000E07EC25F016
:1030100070EF18F0FF0E07EC25F07AEC39F0FF0E98
:1030200007EC25F0AAEC3AF0FF0E07EC25F0AAEC2D
:103030003AF03AEC3BF02AEC3AF0FF0E07EC25F0C0
:10304000FF0E07EC25F09EEC3BF0FF0E07EC25F0A1
:10305000FF0E07EC25F08AEC3AF03AEC3BF09AECE4
:1030600039F0FF0E07EC25F0EAEC39F03AEC3BF0D2
:10307000C30E07EC25F0AEEC24F0400EB7EC24F0C4
:10308000B90EDFEC24F0BD0E07EC25F0BD0E07EC09
:1030900025F0BD0E07EC25F0DB0E07EC25F0FF0E4A
:1030A00007EC25F05AEC3AF0FF0E07EC25F04AEC5D
:1030B0003AF0FF0E07EC25F0AAEC3AF0FF0E07EC11
:1030C00025F08AEC3AF0FF0E07EC25F05AEC3AF0C6
:1030D000FF0E07EC25F02AEC3AF0FF0E07EC25F086
:1030E000ABEC24F0430EB7EC24F0BA0EDFEC24F086
:1030F0001E0E07EC25F0100E07EC25F0100E07EC65
:1031000025F0100E07EC25F0100E07EC25F0ABECC7
:1031100024F0400EB7EC24F0BB0EDFEC24F012B22A
:1031200097EF18F0010E1A5CD8B4B9EF18F0000E42
:1031300007EC25F01AEC38F0000E07EC25F03AEC1D
:1031400039F02AEC3BF06AEC38F0000E07EC25F081
:103150004AEC38F0000E07EC25F08AEC38F0000E4F
:1031600007EC25F05AEC38F0000E07EC25F0D9EF0B
:1031700018F0FF0E07EC25F0CAEC39F0FF0E07EC53
:1031800025F0FAEC3AF03AEC3BF02AEC3AF0FF0E7C
:1031900007EC25F0FAEC39F0FF0E07EC25F04AECCD
:1031A0003AF0FF0E07EC25F01AEC3AF0FF0E07ECB0
:1031B00025F0ABEC24F0430EB7EC24F0BC0EDFECB2
:1031C00024F01E0E07EC25F0100E07EC25F0100E73
:1031D00007EC25F0100E07EC25F0100E07EC25F09B
:1031E000ABEC24F0400EB7EC24F0BD0EDFEC24F085
:1031F00012B200EF19F0020E1A5CD8B443EF19F0C6
:10320000000E07EC25F0FAEC37F0000E07EC25F085
:103210000AEC38F0000E07EC25F01AEC38F0000E3E
:1032200007EC25F0CAEC37F0000E07EC25F0FAECBD
:1032300038F0000E07EC25F06AEC38F0000E07ECD1
:1032400025F0EAEC38F02AEC3BF06AEC38F0000E9E
:1032500007EC25F09AEC38F0000E07EC25F0CAECEC
:1032600037F0AEEC24F0400EB7EC24F0BD0EDFECEE
:1032700024F0000E07EC25F0FAEC37F0000E07EC16
:1032800025F084EF19F0FF0E07EC25F0AAEC39F0D9
:10329000FF0E07EC25F0BAEC39F0FF0E07EC25F035
:1032A000CAEC39F0FF0E07EC25F07AEC39F0FF0E8E
:1032B00007EC25F0BAEC3AF0FF0E07EC25F02AEC0B
:1032C0003AF0FF0E07EC25F0AAEC3AF03AEC3BF0AE
:1032D0002AEC3AF0FF0E07EC25F05AEC3AF0FF0E1C
:1032E00007EC25F07AEC39F0AEEC24F0400EB7ECA8
:1032F00024F0BD0EDFEC24F0FF0E07EC25F0AAEC65
:1033000039F0FF0E07EC25F0ABEC24F0430EB7ECE0
:1033100024F0BE0EDFEC24F01E0E07EC25F0100E9C
:1033200007EC25F0100E07EC25F0100E07EC25F049
:10333000100E07EC25F0ABEC24F04A0EB7EC24F0AD
:10334000BA0EDFEC24F052B226EF1AF012A2AEEF62
:1033500019F0000E1A5CD8B4EAEF19F0000E07EC71
:1033600025F04AEC38F0000E07EC25F08AEC38F036
:10337000000E07EC25F0EAEC38F0000E07EC25F023
:103380000AEC38F0000E07EC25F0CAEC38F0000E1D
:1033900007EC25F06AEC38F0000E07EC25F09AEC0B
:1033A00038F0000E07EC25F0EAEC37F0000E07ECE1
:1033B00025F05AEC38F0AEEC24F0400EB7EC24F0D7
:1033C000BA0EDFEC24F0000E07EC25F02AEC3BF0FF
:1033D000B8EF1AF0FF0E07EC25F0FAEC39F0FF0E0B
:1033E00007EC25F04AEC3AF0FF0E07EC25F0AAECCA
:1033F0003AF0FF0E07EC25F0BAEC39F0FF0E07ECBF
:1034000025F08AEC3AF0FF0E07EC25F02AEC3AF0B2
:10341000FF0E07EC25F05AEC3AF0FF0E07EC25F012
:103420009AEC39F0FF0E07EC25F01AEC3AF0AEEC0E
:1034300024F0400EB7EC24F0BA0EDFEC24F0FF0EBF
:1034400007EC25F02AEC3BF0B8EF1AF012A22EEFB1
:103450001AF0000E1A5CD8B474EF1AF0000E07ECE4
:1034600025F0DAEC38F0000E07EC25F00AEC38F025
:10347000000E07EC25F0AAEC38F0000E07EC25F062
:10348000CAEC37F0000E07EC25F0CAEC38F0000E5D
:1034900007EC25F0CAEC37F0000E07EC25F0EAEC5B
:1034A00038F0000E07EC25F00AEC38F0000E07ECBF
:1034B00025F02AEC3BF0AEEC24F0400EB7EC24F003
:1034C000BA0EDFEC24F052A46DEF1AF0CAEC38F01B
:1034D000000E07EC25F0B8EF1AF06AEC38F0000E99
:1034E00007EC25F0B8EF1AF0FF0E07EC25F09AEC88
:1034F0003AF0FF0E07EC25F0BAEC39F0FF0E07ECBE
:1035000025F06AEC3AF0FF0E07EC25F07AEC39F082
:10351000FF0E07EC25F08AEC3AF0FF0E07EC25F0E1
:103520007AEC39F0FF0E07EC25F0AAEC3AF0FF0E2A
:1035300007EC25F0BAEC39F0FF0E07EC25F03AEC79
:103540003BF0AEEC24F0400EB7EC24F0BA0EDFEC0A
:1035500024F052A4B3EF1AF08AEC3AF0FF0E07EC15
:1035600025F0B8EF1AF02AEC3AF0FF0E07EC25F040
:10357000ABEC24F04A0EB7EC24F0BC0EDFEC24F0E8
:1035800052B0F3EF1AF012A2CBEF1AF0010E1A5C50
:10359000D8B4DFEF1AF0000E07EC25F09AEC38F003
:1035A000000E07EC25F01AEC38F0000E07EC25F0C1
:1035B0001AEC38F0000E07EC25F021EF1BF0FF0E9F
:1035C00007EC25F05AEC3AF0FF0E07EC25F0CAECB8
:1035D00039F0FF0E07EC25F0CAEC39F0FF0E07ECCE
:1035E00025F021EF1BF012A2FBEF1AF0010E1A5C7E
:1035F000D8B40FEF1BF0000E07EC25F09AEC38F072
:10360000000E07EC25F08AEC38F0000E07EC25F0F0
:103610002AEC3BF0000E07EC25F021EF1BF0FF0E2B
:1036200007EC25F05AEC3AF0FF0E07EC25F04AECD7
:103630003AF0FF0E07EC25F02AEC3BF0000E07EC09
:1036400025F0ABEC24F04A0EB7EC24F0BE0EDFEC14
:1036500024F01FB87AEF1BF012A234EF1BF0020E19
:103660001A5CD8B457EF1BF0000E07EC25F0EAEC1B
:1036700037F0000E07EC25F0CAEC37F0000E07EC2F
:1036800025F08AEC38F0000E07EC25F0EAEC37F074
:10369000000E07EC25F00AEC38F0000E07EC25F0E0
:1036A0006AEC38F0000E07EC25F0C6EF1BF0FF0EB9
:1036B00007EC25F09AEC39F0FF0E07EC25F07AECD8
:1036C00039F0FF0E07EC25F04AEC3AF0FF0E07EC5C
:1036D00025F09AEC39F0FF0E07EC25F0BAEC39F042
:1036E000FF0E07EC25F02AEC3AF0FF0E07EC25F070
:1036F000C6EF1BF012A282EF1BF0020E1A5CD8B4C8
:10370000A5EF1BF0000E07EC25F06AEC38F0000E78
:1037100007EC25F09AEC38F0000E07EC25F0CAEC27
:1037200037F0000E07EC25F0FAEC37F0000E07EC4E
:1037300025F02AEC3BF0000E07EC25F02AEC3BF0DC
:10374000000E07EC25F0C6EF1BF0FF0E07EC25F08E
:103750002AEC3AF0FF0E07EC25F05AEC3AF0FF0E97
:1037600007EC25F07AEC39F0FF0E07EC25F0AAEC17
:1037700039F0FF0E07EC25F02AEC3BF0000E07ECC9
:1037800025F02AEC3BF0000E07EC25F078EF01F075
:10379000ABEC24F0410EB7EC24F0B80EDFEC24F0D3
:1037A000700E07EC25F0100E07EC25F0100E07EC5C
:1037B00025F0100E07EC25F0000E07EC25F06AEC62
:1037C00038F0000E07EC25F00AEC38F0000E07EC9C
:1037D00025F00AEC39F0000E07EC25F00AEC38F081
:1037E000000E07EC25F06AEC38F02AEC3BF07AEC9E
:1037F00038F0000E07EC25F00AEC38F0000E07EC6C
:1038000025F0EAEC38F0000E07EC25F00AEC38F071
:10381000AEEC24F0400EB7EC24F0B80EDFEC24F050
:10382000CAEC38F02AEC3BF0DAEC38F0000E07EC8A
:1038300025F00AEC38F0000E07EC25F0EAEC38F041
:10384000000E07EC25F0EAEC38F0000E07EC25F04E
:103850004AEC38F0000E07EC25F08AEC38F0000E48
:1038600007EC25F02AEC38F0000E07EC25F0082ACA
:103870000B0E085CD8B442EF1CF0100E07EC25F0DC
:1038800037EF1CF0086A700E07EC25F0ABEC24F063
:10389000400EB7EC24F0B90EDFEC24F012B656EF70
:1038A0001CF0000E1C5CD8B482EF1CF0000E07EC7C
:1038B00025F0AAEC38F0000E07EC25F00AEC38F001
:1038C000000E07EC25F0CAEC37F0000E07EC25F0EF
:1038D0005AEC38F02AEC3BF03AEC38F0000E07ECEA
:1038E00025F09AEC38F0000E07EC25F06AEC38F081
:1038F000000E07EC25F0FAEC37F0000E07EC25F08F
:10390000ACEF1CF0FF0E07EC25F06AEC3AF0FF0E6E
:1039100007EC25F0BAEC39F0FF0E07EC25F07AEC55
:1039200039F0FF0E07EC25F01AEC3AF03AEC3BF0D8
:10393000EAEC39F0FF0E07EC25F05AEC3AF0FF0EF6
:1039400007EC25F02AEC3AF0FF0E07EC25F0AAEC84
:1039500039F0FF0E07EC25F0ABEC24F0430EB7EC8A
:1039600024F0BA0EDFEC24F01E0E07EC25F0100E4A
:1039700007EC25F0100E07EC25F0100E07EC25F0F3
:10398000100E07EC25F0ABEC24F0400EB7EC24F061
:10399000BD0EDFEC24F012B6D3EF1CF0020E1C5C5F
:1039A000D8B42BEF1DF0000E07EC25F06AEC38F0D0
:1039B000000E07EC25F00AEC38F0000E07EC25F0BD
:1039C0000AEC39F0000E07EC25F00AEC38F0000E96
:1039D00007EC25F06AEC38F02AEC3BF07AEC38F092
:1039E000000E07EC25F0EAEC38F02AEC3BF0CAECCC
:1039F00038F0000E07EC25F0EAEC38F0000E07EC8A
:103A000025F0000E07EC25F0AEEC24F0400EB7ECEC
:103A100024F0BD0EDFEC24F0000E07EC25F0000EC4
:103A200007EC25F0000E07EC25F0EAEC38F0000E6C
:103A300007EC25F04AEC38F0000E07EC25F07AECA4
:103A400038F0000E07EC25F00AEC38F0000E07EC19
:103A500025F081EF1DF0FF0E07EC25F02AEC3AF07F
:103A6000FF0E07EC25F0BAEC39F0FF0E07EC25F05D
:103A7000CAEC3AF0FF0E07EC25F0BAEC39F0FF0E75
:103A800007EC25F02AEC3AF03AEC3BF03AEC3AF04D
:103A9000FF0E07EC25F0AAEC3AF03AEC3BF08AEC8A
:103AA0003AF0FF0E07EC25F0AAEC3AF0FF0E07EC17
:103AB00025F0FF0E07EC25F0AEEC24F0400EB7EC3D
:103AC00024F0BD0EDFEC24F0FF0E07EC25F0FF0E16
:103AD00007EC25F0FF0E07EC25F0AAEC3AF0FF0EFC
:103AE00007EC25F0FAEC39F0FF0E07EC25F03AEC84
:103AF0003AF0FF0E07EC25F0BAEC39F0FF0E07ECB8
:103B000025F0ABEC24F0430EB7EC24F0BE0EDFEC56
:103B100024F01E0E07EC25F0100E07EC25F0100E19
:103B200007EC25F0100E07EC25F0100E07EC25F041
:103B3000ABEC24F0400EB7EC24F0BB0EDFEC24F02D
:103B400012B6A8EF1DF0010E1C5CD8B4D9EF1DF021
:103B5000000E07EC25F0AAEC38F0000E07EC25F07B
:103B60000AEC38F0000E07EC25F0CAEC37F0000E36
:103B700007EC25F05AEC38F02AEC3BF0CAEC38F0B0
:103B8000000E07EC25F00AEC38F0000E07EC25F0EB
:103B9000DAEC38F0000E07EC25F00AEC38F0000EF5
:103BA00007EC25F0EAEC38F0000E07EC25F008EF02
:103BB0001EF0FF0E07EC25F06AEC3AF0FF0E07EC62
:103BC00025F0BAEC39F0FF0E07EC25F07AEC39F06D
:103BD000FF0E07EC25F01AEC3AF03AEC3BF08AECD9
:103BE0003AF0FF0E07EC25F0BAEC39F0FF0E07ECC7
:103BF00025F09AEC3AF0FF0E07EC25F0BAEC39F01C
:103C0000FF0E07EC25F0AAEC3AF0FF0E07EC25F0CA
:103C1000ABEC24F0430EB7EC24F0BC0EDFEC24F048
:103C20001E0E07EC25F0100E07EC25F0100E07EC29
:103C300025F0100E07EC25F0100E07EC25F0ABEC8C
:103C400024F04A0EB7EC24F0BA0EDFEC24F038B0C2
:103C500064EF1EF0000E1C5CD8A432EF1EF012B60A
:103C60004BEF1EF0000E07EC25F03AEC38F0000E9A
:103C700007EC25F09AEC38F0000E07EC25F06AEC22
:103C800038F0000E07EC25F0FAEC37F0000E07ECE8
:103C900025F09CEF1EF0FF0E07EC25F0EAEC39F062
:103CA000FF0E07EC25F05AEC3AF0FF0E07EC25F07A
:103CB0002AEC3AF0FF0E07EC25F0AAEC39F0FF0EE3
:103CC00007EC25F09CEF1EF0000E1C5CD8A46CEFF6
:103CD0001EF012B685EF1EF0000E07EC25F01AEC70
:103CE00038F0000E07EC25F0CAEC38F0000E07ECB7
:103CF00025F00AEC38F0000E07EC25F00AEC38F05D
:103D0000000E07EC25F09CEF1EF0FF0E07EC25F0EF
:103D1000CAEC39F0FF0E07EC25F08AEC3AF0FF0E02
:103D200007EC25F0BAEC39F0FF0E07EC25F0BAEC01
:103D300039F0FF0E07EC25F0ABEC24F04A0EB7EC9F
:103D400024F0BE0EDFEC24F0000E425CD8B4FCEF91
:103D50001EF0010E425CD8B44AEF1FF0020E1C5C4C
:103D6000D8A4B6EF1EF012B6D9EF1EF0000E07EC85
:103D700025F0DAEC38F0000E07EC25F06AEC38F0AC
:103D8000000E07EC25F09AEC38F0000E07EC25F059
:103D90001AEC39F0000E07EC25F02AEC3BF0000E8F
:103DA00007EC25F02AEC3BF0000E07EC25F096EF2F
:103DB0001FF0FF0E07EC25F09AEC3AF0FF0E07EC2F
:103DC00025F02AEC3AF0FF0E07EC25F05AEC3AF019
:103DD000FF0E07EC25F0DAEC3AF0FF0E07EC25F0C9
:103DE0002AEC3BF0000E07EC25F02AEC3BF0000E2D
:103DF00007EC25F096EF1FF0020E1C5CD8A404EF30
:103E00001FF012B627EF1FF0000E07EC25F01AEC9A
:103E100038F0000E07EC25F0CAEC37F0000E07EC86
:103E200025F0DAEC38F0000E07EC25F0EAEC38F07B
:103E3000000E07EC25F02AEC3BF0000E07EC25F015
:103E40002AEC3BF0000E07EC25F096EF1FF0FF0E7A
:103E500007EC25F0CAEC39F0FF0E07EC25F07AEC00
:103E600039F0FF0E07EC25F09AEC3AF0FF0E07EC64
:103E700025F0AAEC3AF0FF0E07EC25F02AEC3BF017
:103E8000000E07EC25F02AEC3BF0000E07EC25F0C5
:103E900096EF1FF0020E1C5CD8A452EF1FF012B672
:103EA00075EF1FF0000E07EC25F08AEC38F0000EDD
:103EB00007EC25F09AEC38F0000E07EC25F0CAEC80
:103EC00038F0000E07EC25F07AEC38F0000E07EC25
:103ED00025F0CAEC37F0000E07EC25F06AEC38F05C
:103EE000000E07EC25F096EF1FF0FF0E07EC25F013
:103EF0004AEC3AF0FF0E07EC25F05AEC3AF0FF0ED0
:103F000007EC25F08AEC3AF0FF0E07EC25F03AECCE
:103F10003AF0FF0E07EC25F07AEC39F0FF0E07ECD3
:103F200025F02AEC3AF0FF0E07EC25F0ABEC24F07C
:103F30004A0EB7EC24F0BC0EDFEC24F038B203EFED
:103F400020F0010E1C5CD8A4A9EF1FF012B6D6EF2A
:103F50001FF0000E07EC25F0EAEC38F0000E07EC3D
:103F600025F04AEC38F0000E07EC25F07AEC38F03A
:103F7000000E07EC25F00AEC38F02AEC3BF09AEC46
:103F800038F0000E07EC25F0FAEC38F0000E07ECE4
:103F900025F0EAEC38F0000E07EC25F0000E07ECF7
:103FA00025F0000E07EC25F063EF20F0FF0E07EC84
:103FB00025F0AAEC3AF0FF0E07EC25F0FAEC39F008
:103FC000FF0E07EC25F03AEC3AF0FF0E07EC25F077
:103FD000BAEC39F03AEC3BF05AEC3AF0FF0E07EC51
:103FE00025F0BAEC3AF0FF0E07EC25F0AAEC3AF017
:103FF000FF0E07EC25F0000E07EC25F0000E07EC95
:1040000025F063EF20F0010E1C5CD8A40BEF20F02C
:1040100012B638EF20F0000E07EC25F0FAEC37F07E
:10402000000E07EC25F00AEC38F0000E07EC25F046
:10403000EAEC37F0000E07EC25F0CAEC38F0000E81
:1040400007EC25F00AEC38F0000E07EC25F0CAEC7E
:1040500037F0000E07EC25F0DAEC38F0000E07EC34
:1040600025F00AEC38F0000E07EC25F063EF20F0A5
:10407000FF0E07EC25F0AAEC39F0FF0E07EC25F057
:10408000BAEC39F0FF0E07EC25F09AEC39F0FF0E90
:1040900007EC25F08AEC3AF0FF0E07EC25F0BAECBD
:1040A00039F0FF0E07EC25F07AEC39F0FF0E07EC43
:1040B00025F09AEC3AF0FF0E07EC25F0BAEC39F057
:1040C000FF0E07EC25F078EF01F0ABEC24F0410E89
:1040D000B7EC24F0B80EDFEC24F0700E07EC25F0FE
:1040E000100E07EC25F0100E07EC25F0100E07EC73
:1040F00025F0000E07EC25F00AEC38F0000E07EC76
:1041000025F00AEC38F0000E07EC25F0AAEC38F0A8
:10411000000E07EC25F0CAEC38F0000E07EC25F095
:104120009AEC38F0000E07EC25F07AEC38F0000E2F
:1041300007EC25F02AEC3BF01AEC39F0000E07EC06
:1041400025F0CAEC38F0000E07EC25F04AEC38F008
:10415000AEEC24F0400EB7EC24F0B80EDFEC24F007
:10416000000E07EC25F0EAEC38F0000E07EC25F025
:104170000AEC38F0000E07EC25F0082A320E085C35
:10418000D8B4C8EF20F0100E07EC25F0BDEF20F0FA
:10419000086A700E07EC25F0ABEC24F0460EB7EC85
:1041A00024F0B90EDFEC24F012B45FEF23F0DAEC68
:1041B00038F0000E07EC25F00AEC38F0000E07ECA2
:1041C00025F06AEC38F0000E07EC25F00AEC38F028
:1041D000000E07EC25F0EAEC37F0000E07EC25F0B6
:1041E000EAEC38F0000E07EC25F02AEC3BF0CAECC4
:1041F00037F0000E07EC25F0FAEC37F0000E07EC74
:1042000025F0FAEC37F0AEEC24F0400EB7EC24F0D9
:10421000B90EDFEC24F0000E07EC25F0CAEC38F004
:10422000000E07EC25F00AEC38F0000E07EC25F044
:10423000DAEC38F0000E07EC25F0DAEC38F0000E7E
:1042400007EC25F0ABEC24F04A0EB7EC24F0BB0EE3
:10425000DFEC24F0000E1B5CD8B443EF21F0000E1D
:1042600007EC25F0FAEC34F0000E07EC25F04AECF0
:1042700035F0000E07EC25F0FAEC37F0000E07ECF5
:1042800025F055EF21F0FF0E07EC25F09AEC35F004
:10429000FF0E07EC25F0EAEC35F0FF0E07EC25F0F9
:1042A000AAEC39F0FF0E07EC25F0ABEC24F0670E1A
:1042B000B7EC24F0BB0EDFEC24F0010E1B5CD8B48D
:1042C00076EF21F0000E07EC25F0FAEC34F0000E4A
:1042D00007EC25F05AEC35F0000E07EC25F0FAEC6F
:1042E00037F0000E07EC25F088EF21F0FF0E07EC09
:1042F00025F09AEC35F0FF0E07EC25F0FAEC35F0DE
:10430000FF0E07EC25F0AAEC39F0FF0E07EC25F0C4
:10431000AEEC24F0440EB7EC24F0BB0EDFEC24F03E
:10432000020E1B5CD8B4A9EF21F0000E07EC25F0BB
:10433000FAEC34F0000E07EC25F06AEC35F0000ED4
:1043400007EC25F0FAEC37F0000E07EC25F0BBEF98
:1043500021F0FF0E07EC25F09AEC35F0FF0E07EC8C
:1043600025F00AEC36F0FF0E07EC25F0AAEC39F048
:10437000FF0E07EC25F0AEEC24F0610EB7EC24F054
:10438000BB0EDFEC24F0030E1B5CD8B4DCEF21F095
:10439000000E07EC25F0FAEC34F0000E07EC25F0E7
:1043A0007AEC35F0000E07EC25F0FAEC37F0000E51
:1043B00007EC25F0EEEF21F0FF0E07EC25F09AEC6C
:1043C00035F0FF0E07EC25F01AEC36F0FF0E07EC87
:1043D00025F0AAEC39F0FF0E07EC25F0ABEC24F049
:1043E0004A0EB7EC24F0BC0EDFEC24F0040E1B5C8C
:1043F000D8B40FEF22F0000E07EC25F00AEC35F0F0
:10440000000E07EC25F0EAEC34F0000E07EC25F086
:10441000FAEC37F0000E07EC25F021EF22F0FF0E4A
:1044200007EC25F0AAEC35F0FF0E07EC25F08AEC3E
:1044300035F0FF0E07EC25F0AAEC39F0FF0E07EC83
:1044400025F0ABEC24F0670EB7EC24F0BC0EDFECEB
:1044500024F0050E1B5CD8B442EF22F0000E07ECEE
:1044600025F00AEC35F0000E07EC25F0FAEC34F0FC
:10447000000E07EC25F0FAEC37F0000E07EC25F003
:1044800054EF22F0FF0E07EC25F0AAEC35F0FF0EFA
:1044900007EC25F09AEC35F0FF0E07EC25F0AAECBE
:1044A00039F0FF0E07EC25F0ABEC24F04A0EB7EC28
:1044B00024F0BD0EDFEC24F0060E1B5CD8B48DEFAB
:1044C00022F0000E07EC25F09AEC38F0000E07EC15
:1044D00025F0EAEC38F0000E07EC25F03AEC38F065
:1044E000000E07EC25F00AEC38F0000E07EC25F082
:1044F000CAEC38F02AEC3BF0DAEC38F0000E07ECAE
:1045000025F00AEC38F0000E07EC25F0EAEC38F064
:10451000000E07EC25F0B7EF22F0FF0E07EC25F0B8
:104520005AEC3AF0FF0E07EC25F0AAEC3AF0FF0E39
:1045300007EC25F0EAEC39F0FF0E07EC25F0BAECB9
:1045400039F0FF0E07EC25F08AEC3AF03AEC3BF03C
:104550009AEC3AF0FF0E07EC25F0BAEC39F0FF0EBA
:1045600007EC25F0AAEC3AF0FF0E07EC25F0AEECD4
:1045700024F0440EB7EC24F0BD0EDFEC24F0070E5F
:104580001B5CD8B4EAEF22F0000E07EC25F06AECD1
:1045900038F0000E07EC25F00AEC39F02AEC3BF07D
:1045A0007AEC38F0000E07EC25F0EAEC38F02AEC53
:1045B0003BF0DAEC38F0000E07EC25F00AEC38F0AE
:1045C000000E07EC25F0EAEC38F0000E07EC25F0C1
:1045D0000EEF23F0FF0E07EC25F02AEC3AF0FF0E69
:1045E00007EC25F0CAEC3AF03AEC3BF03AEC3AF042
:1045F000FF0E07EC25F0AAEC3AF03AEC3BF09AEC0F
:104600003AF0FF0E07EC25F0BAEC39F0FF0E07EC9C
:1046100025F0AAEC3AF0FF0E07EC25F0ABEC24F005
:104620004A0EB7EC24F0BF0EDFEC24F0080E1B5C42
:10463000D8B43DEF23F0000E07EC25F0CAEC37F0BC
:10464000000E07EC25F06AEC38F0000E07EC25F0C0
:104650006AEC38F02AEC3BF0DAEC38F0000E07ECAC
:1046600025F00AEC38F0000E07EC25F0EAEC38F003
:10467000000E07EC25F05DEF23F0FF0E07EC25F0B0
:104680007AEC39F0FF0E07EC25F02AEC3AF0FF0E39
:1046900007EC25F02AEC3AF03AEC3BF09AEC3AF0D1
:1046A000FF0E07EC25F0BAEC39F0FF0E07EC25F011
:1046B000AAEC3AF0FF0E07EC25F078EF01F0000EBF
:1046C0001B5CD8A47EEF23F0C2EC3BF0FAEC34F094
:1046D000000E07EC25F04AEC35F0000E07EC25F053
:1046E00072EF23F0AEEC24F0400EB7EC24F0B90EDC
:1046F000DFEC24F0FAEC37F047EF24F0010E1B5CFE
:10470000D8A491EF23F0C2EC3BF0FAEC34F0000EA9
:1047100007EC25F05AEC35F0000E07EC25F072EFAF
:1047200023F0020E1B5CD8A4A4EF23F0C2EC3BF0F4
:10473000FAEC34F0000E07EC25F06AEC35F0000ED0
:1047400007EC25F072EF23F0030E1B5CD8A4B7EF43
:1047500023F0C2EC3BF0FAEC34F0000E07EC25F04D
:104760007AEC35F0000E07EC25F072EF23F0040E22
:104770001B5CD8A4CAEF23F0C2EC3BF00AEC35F086
:10478000000E07EC25F0EAEC34F0000E07EC25F003
:1047900072EF23F0050E1B5CD8A4DDEF23F0C2EC12
:1047A0003BF00AEC35F0000E07EC25F0FAEC34F0A3
:1047B000000E07EC25F072EF23F0060E1B5CD8A468
:1047C00008EF24F09AEC38F0000E07EC25F0EAEC44
:1047D00038F0000E07EC25F03AEC38F0000E07EC4C
:1047E00025F00AEC38F0000E07EC25F0CAEC38F0A2
:1047F0002AEC3BF0DAEC38F0000E07EC25F00AEC7E
:1048000038F0000E07EC25F0EAEC38F047EF24F022
:10481000070E1B5CD8A42DEF24F06AEC38F0000ED4
:1048200007EC25F00AEC39F02AEC3BF07AEC38F092
:10483000000E07EC25F0EAEC38F02AEC3BF0DAEC5D
:1048400038F0000E07EC25F00AEC38F0000E07EC0B
:1048500025F0EAEC38F047EF24F0CAEC37F0000E10
:1048600007EC25F06AEC38F0000E07EC25F06AEC56
:1048700038F02AEC3BF0DAEC38F0000E07EC25F0CB
:104880000AEC38F0000E07EC25F0EAEC38F0ABEC5F
:1048900024F0670EB7EC24F0BC0EDFEC24F01FBE52
:1048A00066EF24F0000E07EC25F03AEC39F0000E2C
:1048B00007EC25F00AEC38F0000E07EC25F0DAECF6
:1048C00038F0000E07EC25F078EF24F0FF0E07EC2F
:1048D00025F0FAEC3AF0FF0E07EC25F0BAEC39F0CF
:1048E000FF0E07EC25F09AEC3AF0FF0E07EC25F0EE
:1048F000AEEC24F0440EB7EC24F0BC0EDFEC24F058
:104900001FBE97EF24F0FF0E07EC25F04AEC3AF0BB
:10491000FF0E07EC25F03AEC3BF0FF0E07EC25F01C
:104920005AEC3AF0FF0E07EC25F0A9EF24F0000E48
:1049300007EC25F08AEC38F0000E07EC25F02AECA5
:104940003BF0000E07EC25F09AEC38F0000E07EC77
:1049500025F078EF01F08C888C9A12008C988C8A64
:1049600012008C888C8A12008C988C9A1200016E2E
:1049700032EC25F001508B6E8C928C900000000080
:104980000000000000000000000000000000000027
:104990008C84000000000000000000000000000007
:1049A0000000000000008C940000000000000000E7
:1049B0000000000000000000000000001200026E75
:1049C00032EC25F002508B6E8C928C90000000002F
:1049D00000000000000000000000000000000000D7
:1049E0008C840000000000000000000000000000B7
:1049F0000000000000008C94000000000000000097
:104A00000000000000000000000000001200006E26
:104A100032EC25F012BE70EC25F000508B6E8C92BB
:104A20008C8000000000000000000000000000007A
:104A30000000000000008C84000000000000000066
:104A40000000000000000000000000008C94000046
:104A50000000000000000000000000000000000056
:104A6000000012000F01FF0E946E00018C828C90EA
:104A70000000000000000000000000000000000036
:104A8000000000008C840000000000000000000016
:104A90000000000000000000000000000000000016
:104AA00000000000000000000000000000008C94E6
:104AB00000000000000000000000000000000000F6
:104AC000000000000000000000000000000082BEA6
:104AD00042EF25F08C920F01000E946E000112003F
:104AE000000E205CD8B495EF25F0010E205CD8B400
:104AF000AEEF25F0020E205CD8B4C5EF25F0030E12
:104B0000205CD8B4DAEF25F0040E205CD8B4EDEFC9
:104B100025F0050E205CD8B4FEEF25F0060E205CD3
:104B2000D8B40DEF26F01AEF26F01FB0A3EF25F052
:104B30000042004200420042004200420042010E98
:104B400000161AEF26F000460046004600460046D2
:104B500000460046800E00161AEF26F01FB0BBEF8D
:104B600025F0004200420042004200420042030E93
:104B700000161AEF26F000460046004600460046A2
:104B80000046C00E00161AEF26F01FB0D1EF25F038
:104B900000420042004200420042070E00161AEF97
:104BA00026F000460046004600460046E00E00168D
:104BB0001AEF26F01FB0E5EF25F000420042004258
:104BC00000420F0E00161AEF26F00046004600467F
:104BD0000046F00E00161AEF26F01FB0F7EF25F092
:104BE0000042004200421F0E00161AEF26F0004657
:104BF00000460046F80E00161AEF26F01FB007EF29
:104C000026F0004200423F0E00161AEF26F0004642
:104C10000046FC0E00161AEF26F01FB015EF26F026
:104C200000427F0E00161AEF26F00046FE0E001618
:104C30001AEF26F01200B1EC24F0400EB7EC24F08D
:104C4000B80EDFEC24F0000E07EC25F0012A800EF0
:104C5000015CD8A423EF26F0022AE0EC24F0400EF9
:104C6000B7EC24F0C00E025CD8A423EF26F01200AB
:104C70008098479E47AE40EF26F0808441EF26F0B3
:104C80008094000000000000818A00000000000005
:104C9000819A082A080E085CD8B452EF26F04746DD
:104CA0003AEF26F0086A45AE59EF26F080845AEFB5
:104CB00026F08094000000000000818A00000000BF
:104CC0000000819A082A080E085CD8B46BEF26F021
:104CD000454653EF26F0086A808812008098478E78
:104CE00047AE76EF26F0808477EF26F080940000C0
:104CF00000000000818A000000000000819A082A5C
:104D0000080E085CD8B488EF26F0474670EF26F00E
:104D1000086A818A00000000000081A893EF26F055
:104D2000468094EF26F04690819A00000000000033
:104D3000082A080E085CD8B4A1EF26F0464689EF91
:104D400026F0086A808846501200106E000E105C33
:104D5000D8A4C3EF26F005B8B4EF26F005BAB8EF33
:104D600026F04AEC34F012002AEC3BF0058C1200DD
:104D700005BCBFEF26F0059C4AEC34F01200059C00
:104D80002AEC3BF01200010E105CD8A4CBEF26F009
:104D90005AEC34F01200020E105CD8A4D3EF26F0C7
:104DA0006AEC34F01200030E105CD8A4DBEF26F09E
:104DB0007AEC34F01200040E105CD8A4E3EF26F075
:104DC0008AEC34F01200050E105CD8A4EBEF26F04C
:104DD0009AEC34F01200060E105CD8A4F3EF26F023
:104DE000AAEC34F01200070E105CD8A4FBEF26F0FA
:104DF000BAEC34F01200080E105CD8A403EF27F0D0
:104E0000CAEC34F01200DAEC34F01200106E000E2E
:104E1000105CD8A40FEF27F0EAEC34F01200010E7A
:104E2000105CD8A417EF27F0FAEC34F01200020E51
:104E3000105CD8A41FEF27F00AEC35F01200030E27
:104E4000105CD8A427EF27F01AEC35F01200040EFE
:104E5000105CD8A42FEF27F02AEC35F01200050ED5
:104E6000105CD8A437EF27F03AEC35F01200060EAC
:104E7000105CD8A43FEF27F04AEC35F01200070E83
:104E8000105CD8A447EF27F05AEC35F01200080E5A
:104E9000105CD8A44FEF27F06AEC35F012007AECE2
:104EA00035F01200106E000E105CD8A45BEF27F0F6
:104EB0008AEC35F01200010E105CD8A463EF27F0E5
:104EC0009AEC35F01200020E105CD8A46BEF27F0BC
:104ED000AAEC35F01200030E105CD8A473EF27F093
:104EE000BAEC35F01200040E105CD8A47BEF27F06A
:104EF000CAEC35F01200050E105CD8A483EF27F041
:104F0000DAEC35F01200060E105CD8A48BEF27F017
:104F1000EAEC35F01200070E105CD8A493EF27F0EE
:104F2000FAEC35F01200080E105CD8A49BEF27F0C5
:104F30000AEC36F012001AEC36F01200062A0A0EBD
:104F4000065CD8A49EEF27F0066A1200062AFF0E20
:104F5000065CD8A4A6EF27F0066A072A550E075C60
:104F6000D8A4A6EF27F0066A076A1200062AFF0EE9
:104F7000065CD8A4B6EF27F0066A072AFF0E075C86
:104F8000D8A4B6EF27F0066A076A1200100E476E23
:104F90004850456E38EC26F0110E476E4950456E6C
:104FA00038EC26F0120E476E4A50456E38EC26F06B
:104FB000130E476E4B50456E38EC26F0140E476EBC
:104FC0004C50456E38EC26F0150E476E4D50456E30
:104FD00038EC26F01200ABEC24F0400EB7EC24F0D5
:104FE000BF0EDFEC24F0FAEC37F0000E07EC25F0F2
:104FF000CAEC37F0000E07EC25F0EAEC37F0000EB3
:1050000007EC25F0FAEC34F0000E07EC25F05AEC32
:1050100035F0000E07EC25F07AEC35F0000E07ECC9
:1050200025F00AEC35F02AEC3BF0CAEC38F0000E23
:1050300007EC25F00AEC38F0000E07EC25F00AEC3E
:1050400039F0AEEC24F0400EB7EC24F0BF0EDFECEC
:1050500024F0400E07EC25F0000E07EC25F0FAECEA
:1050600034F0000E07EC25F0400E07EC25F0000EA2
:1050700007EC25F0EAEC34F0000E07EC25F0400ECA
:10508000036E7F0E046EABEC24F00350B7EC24F0FB
:10509000BC0EDFEC24F0010E07EC25F0AEEC24F0A2
:1050A0000450B7EC24F0BC0EDFEC24F0010E07EC4A
:1050B00025F0032A0406A6EC27F0A6EC27F0800EC4
:1050C000035CD8A443EF28F0B6EC27F0B6EC27F049
:1050D000B6EC27F0B6EC27F0B6EC27F0B6EC27F0EC
:1050E000B6EC27F0B6EC27F0B6EC27F0A6EC27F0EC
:1050F000400E036E7F0E046EABEC24F00350B7EC51
:1051000024F0BC0EDFEC24F0000E07EC25F0AEEC32
:1051100024F00450B7EC24F0BC0EDFEC24F0000EB9
:1051200007EC25F0032A0406A6EC27F0A6EC27F0EE
:10513000800E035CD8A47CEF28F0128EB6EC27F02A
:10514000B6EC27F0B6EC27F0B6EC27F0B6EC27F07B
:10515000B6EC27F0B6EC27F0A6EC27F01F80C6ECE3
:1051600027F0ABEC24F04A0EB7EC24F0BB0EDFECDA
:1051700024F07AEC36F0000E07EC25F0100E07EC68
:1051800025F0100E07EC25F0100E07EC25F0100EA0
:1051900007EC25F0100E07EC25F0000E07EC25F0CB
:1051A000FAEC36F0000E07EC25F02AEC3BF0000E8E
:1051B00007EC25F06AEC36F0000E07EC25F0FAEC6F
:1051C00036F0000E07EC25F08AEC36F0000E07EC06
:1051D00025F0AAEC36F0000E07EC25F0FAEC36F0DC
:1051E000000E07EC25F0AEEC24F0400EB7EC24F0F6
:1051F000BB0EDFEC24F06AEC36F0000E07EC25F075
:105200006AEC36F0000E07EC25F03AEC37F0000EB1
:1052100007EC25F0AAEC36F0000E07EC25F0FAECCE
:1052200036F0000E07EC25F08AEC36F0000E07ECA5
:1052300025F01F90ABEC24F0560EB7EC24F0BC0E1A
:10524000DFEC24F02AEC36F0000E07EC25F06AECD7
:1052500037F0000E07EC25F05AEC36F0000E07ECA4
:1052600025F0AAEC36F0000E07EC25F00AEC37F03A
:10527000000E07EC25F02AEC3BF0000E07EC25F0C1
:10528000DAEC36F0000E07EC25F0AEEC24F0400E20
:10529000B7EC24F0BC0EDFEC24F02AEC36F0000E64
:1052A00007EC25F03AEC36F0000E07EC25F00AEC9E
:1052B00037F0000E07EC25F03AEC37F0000E07EC63
:1052C00025F02AEC36F0000E07EC25F05AEC37F00A
:1052D000000E07EC25F00AEC37F0000E07EC25F085
:1052E0003AEC37F0000E07EC25F0AAEC37F0000E90
:1052F00007EC25F0202A080E205CD8A49EEF28F0A9
:10530000129E206AB6EC27F0B6EC27F0B6EC27F038
:10531000B6EC27F0B6EC27F0B6EC27F0B6EC27F0A9
:10532000B6EC27F0B6EC27F0B6EC27F0B6EC27F099
:10533000B6EC27F0B6EC27F0B6EC27F0B6EC27F089
:10534000B6EC27F0B6EC27F0B6EC27F0B6EC27F079
:10535000B6EC27F0B6EC27F0B6EC27F0B6EC27F069
:10536000B6EC27F0B6EC27F0B6EC27F0B6EC27F059
:10537000B6EC27F0B6EC27F0B6EC27F0B6EC27F049
:10538000B6EC27F0B6EC27F0B6EC27F0B6EC27F039
:10539000B6EC27F0B6EC27F0B6EC27F0B6EC27F029
:1053A000B6EC27F0B6EC27F0B6EC27F0B6EC27F019
:1053B000B6EC27F0B6EC27F0B6EC27F0B6EC27F009
:1053C000B6EC27F0B6EC27F0B6EC27F0B6EC27F0F9
:1053D000B6EC27F0B6EC27F0B6EC27F0B6EC27F0E9
:1053E000B6EC27F0B6EC27F0B6EC27F0B6EC27F0D9
:1053F000B6EC27F0B6EC27F0B6EC27F0B6EC27F0C9
:10540000B6EC27F0B6EC27F0B6EC27F0B6EC27F0B8
:10541000B6EC27F0B6EC27F0B6EC27F0B6EC27F0A8
:10542000B6EC27F0B6EC27F0B6EC27F0B6EC27F098
:10543000B6EC27F0B6EC27F0B6EC27F0B6EC27F088
:10544000B6EC27F0B6EC27F0B6EC27F0B6EC27F078
:10545000B6EC27F0B6EC27F0B6EC27F0B6EC27F068
:10546000B6EC27F0B6EC27F0B6EC27F0B6EC27F058
:10547000B6EC27F0B6EC27F0B6EC27F0B6EC27F048
:10548000B6EC27F0B6EC27F0B6EC27F0B6EC27F038
:10549000B6EC27F0B6EC27F0B6EC27F0B6EC27F028
:1054A000B6EC27F0B6EC27F0B6EC27F01BEC26F0B4
:1054B000B6EC27F0B6EC27F0B6EC27F0B6EC27F008
:1054C000B6EC27F0B6EC27F0B6EC27F0B6EC27F0F8
:1054D000B6EC27F0B6EC27F0120081B27BEF2AF091
:1054E000460E575CD8B477EF2AF0572A1200576A55
:1054F000586A128C1200576A81A289EF2AF0640E52
:10550000565CD8B487EF2AF0562A7CEF2AF0566A08
:105510001200566A81B49AEF2AF0140E565CD8B481
:1055200095EF2AF0562A8AEF2AF0566A556A586A89
:10553000128C1200566A81A0A1EF2AF0588EA3EFB8
:105540002AF0589E0000552A080E555CD8B4ACEFDE
:105550002AF058428AEF2AF0556A81B4BDEF2AF04A
:10556000140E565CD8B4B8EF2AF0562AADEF2AF0E4
:10557000566A556A586A128C1200566A81A0C4EFA6
:105580002AF0598EC6EF2AF0599E0000552A080EBF
:10559000555CD8B4CFEF2AF05942ADEF2AF0556AE6
:1055A00081B4E0EF2AF0140E565CD8B4DBEF2AF099
:1055B000562AD0EF2AF0566A556A586A128C1200A1
:1055C000566A81A0E7EF2AF05A8EE9EF2AF05A9E38
:1055D0000000552A080E555CD8B4F2EF2AF05A4262
:1055E000D0EF2AF0556A81B403EF2BF0140E565C0D
:1055F000D8B4FEEF2AF0562AF3EF2AF0566A556A1D
:10560000586A128C1200566A81A00AEF2BF05B8E4A
:105610000CEF2BF05B9E0000552A080E555CD8B4A9
:1056200015EF2BF05B42F3EF2AF0556A81B426EFB9
:105630002BF0140E565CD8B421EF2BF0562A16EF3F
:105640002BF0566A556A586A128C1200566A81A06D
:105650002DEF2BF05C8E2FEF2BF05C9E0000552A77
:10566000080E555CD8B438EF2BF05C4216EF2BF0E7
:10567000556A81B449EF2BF0140E565CD8B444EF50
:105680002BF0562A39EF2BF0566A556A586A128C5D
:105690001200566A81A050EF2BF05D8E52EF2BF076
:1056A0005D9E0000552A080E555CD8B45BEF2BF0C8
:1056B0005D4239EF2BF0556A81B46CEF2BF0140E7C
:1056C000565CD8B467EF2BF0562A5CEF2BF0566A85
:1056D000556A586A128C1200566A81A073EF2BF03B
:1056E0005E8E75EF2BF05E9E0000552A080E555C0D
:1056F000D8B47EEF2BF05E425CEF2BF0556AD40EEF
:10570000585CD8A487EF2BF0129C88EF2BF0128CFA
:10571000120051A0120012BC12005EAE12004CAA80
:1057200099EF2BF04C9A140E476E4C50456E38ECA6
:1057300026F05DBE0AEF2CF05C505F6E5F965F94C2
:105740004A50700B606F800E5F5CD8A4B1EF2BF0F5
:10575000000E605DD8B412004A9C4A9A4A9811EF34
:105760002CF0400E5F5CD8A4BFEF2BF0100E605DF4
:10577000D8B412004A9C4A9A4A8811EF2CF0000EC5
:105780005F5CD8A4CDEF2BF0200E605DD8B4120082
:105790004A9C4A8A4A9811EF2CF0930E5F5CD8A479
:1057A000DBEF2BF0400E605DD8B412004A8C4A9AB1
:1057B0004A9811EF2CF0530E5F5CD8B4E7EF2BF052
:1057C000130E5F5CD8B4E7EF2BF0F0EF2BF0500E28
:1057D000605DD8B412004A8C4A9A4A8811EF2CF0C6
:1057E000900E5F5CD8B401EF2CF0500E5F5CD8B423
:1057F00001EF2CF0100E5F5CD8B401EF2CF00AEF33
:105800002CF0300E605DD8B412004A9C4A8A4A8857
:1058100011EF2CF0700E605DD8B412004A8C4A8AE9
:105820004A88120E476E4A50456E38EC26F0120038
:10583000096E640E095ED8A021EF2CF00A2A19EF38
:105840002CF0640E09260A0E095ED8A02BEF2CF06E
:105850000B2A23EF2CF00A0E0926010E095ED8A0B0
:1058600035EF2CF00C2A2DEF2CF012000D6E100EDF
:105870000D5ED8A03FEF2CF00B2A37EF2CF0100E66
:105880000D26010E0D5ED8A049EF2CF00C2A41EF39
:105890002CF0120005880A50A5EC26F0000E07EC4B
:1058A00025F00598058A0B50A5EC26F0000E07ECB4
:1058B00025F0059A0C50A5EC26F0000E07EC25F01B
:1058C0000A6A0B6A0C6A12000A5006EC27F0000EF6
:1058D00007EC25F00B5006EC27F0000E07EC25F046
:1058E0000C5006EC27F0000E07EC25F00A6A0B6A54
:1058F0000C6A12000A5052EC27F0FF0E07EC25F05C
:105900000B5052EC27F0FF0E07EC25F00C5052EC38
:1059100027F0FF0E07EC25F00A6A0B6A0C6A1200EA
:10592000136E182A090E185CD8B4A6EF2CF013BE1B
:105930009EEF2CF0EAEC34F0A0EF2CF0FAEC34F00F
:10594000000E07EC25F0134691EF2CF0186A1200B8
:10595000136E080E185CD8B4E5EF2CF013BECAEF36
:105960002CF018501D5CD8B4C0EF2CF0000E07ECE2
:1059700025F0EAEC34F0000E07EC25F0E1EF2CF016
:10598000FF0E07EC25F08AEC35F0FF0E07EC25F052
:10599000E1EF2CF018501D5CD8B4D9EF2CF0000EBC
:1059A00007EC25F0FAEC34F0000E07EC25F0E1EFFF
:1059B0002CF0FF0E07EC25F09AEC35F0FF0E07EC0B
:1059C00025F0182A1346A9EF2CF0186A120080AEB1
:1059D000EDEF2CF02180EEEF2CF0219080ACF4EF75
:1059E0002CF02182F5EF2CF02192030E215CD8B42B
:1059F000118C000E215CD8A44AEF2EF011AC4AEFB6
:105A00002EF0119C020E225CD8A4A8EF2DF0000EFF
:105A1000145CD8B422EF2DF0010E145CD8B42CEF36
:105A20002DF0020E145CD8B430EF2DF0030E145C90
:105A3000D8B449EF2DF0040E145CD8B477EF2DF0F4
:105A40009AEF2DF04CBA4AEF2EF04CB84AEF2EF0F8
:105A5000B9EC2EF04AEF2EF02CEC2FF04AEF2EF09E
:105A600012B03BEF2DF0000E195CD8B44AEF2EF0C7
:105A700019064AEF2EF01FBA46EF2DF0080E1D5CF6
:105A8000D8B44AEF2EF01D2A4AEF2EF01F8C4AEFB1
:105A90002EF012B256EF2DF0000E1A5CD8B44AEF79
:105AA0002EF01A064AEF2EF04AEF2EF0000E1A5C86
:105AB000D8B462EF2DF0010E1A5CD8B46FEF2DF060
:105AC00073EF2DF052A24AEF2EF052A46BEF2DF09F
:105AD00052944AEF2EF0529452924AEF2EF052B066
:105AE00052904AEF2EF01FB81F984AEF2EF012B6D0
:105AF00082EF2DF0000E1C5CD8B44AEF2EF01C068D
:105B00004AEF2EF0000E1C5CD8A48AEF2DF03880EE
:105B10004AEF2EF0010E1C5CD8A492EF2DF03892C3
:105B20004AEF2EF0020E425CD8B44AEF2EF0422A21
:105B30004AEF2EF012B4A5EF2DF0000E1B5CD8B486
:105B40004AEF2EF01B064AEF2EF01F8E4AEF2EF082
:105B5000010E225CD8A44AEF2EF0000E145CD8B4DB
:105B6000C8EF2DF0010E145CD8B4D2EF2DF0020E68
:105B7000145CD8B4D6EF2DF0030E145CD8B4EFEF5C
:105B80002DF0040E145CD8B41BEF2EF03EEF2EF077
:105B90004CBA4AEF2EF04CB84AEF2EF051EC2EF0F2
:105BA0004AEF2EF021EC2FF04AEF2EF012B0E1EF89
:105BB0002DF0050E195CD8B44AEF2EF0192A4AEFE1
:105BC0002EF01FBAECEF2DF0000E1D5CD8B44AEF9A
:105BD0002EF01D064AEF2EF01F9C4AEF2EF012B257
:105BE000FCEF2DF0020E1A5CD8B44AEF2EF01A2A00
:105BF0004AEF2EF04AEF2EF0000E1A5CD8B408EFF0
:105C00002EF0010E1A5CD8B413EF2EF017EF2EF021
:105C100052B20FEF2EF0528252944AEF2EF052A45D
:105C200052844AEF2EF052A052804AEF2EF01FA865
:105C30001F884AEF2EF012B626EF2EF0020E1C5CE3
:105C4000D8B44AEF2EF01C2A4AEF2EF0000E1C5C4E
:105C5000D8A42EEF2EF038904AEF2EF0010E1C5CE7
:105C6000D8A436EF2EF038824AEF2EF0000E425CB8
:105C7000D8B44AEF2EF042064AEF2EF012B449EFA4
:105C80002EF0080E1B5CD8B44AEF2EF01B2A4AEF08
:105C90002EF01F9E2150226EFF0E355CD8A4352AAF
:105CA00012004AAE1200010E355CD8B05CEF2EF047
:105CB0001A0E366E82EF2EF00F0E355CD8B065EFFF
:105CC0002EF0140E366E82EF2EF01E0E355CD8B01C
:105CD0006EEF2EF00C0E366E82EF2EF02D0E355C30
:105CE000D8B077EF2EF0060E366E82EF2EF03C0E17
:105CF000355CD8B080EF2EF0030E366E82EF2EF0BA
:105D0000010E366E51A288EF2EF051B497EF2EF0AF
:105D10003650396EFF0E485CD8B497EF2EF0482A03
:105D20003906000E395CD8A48AEF2EF0356A51A2EC
:105D30009DEF2EF051A4ACEF2EF03650396EFF0ED1
:105D4000495CD8B4ACEF2EF0492A3906000E395C14
:105D5000D8A49FEF2EF0356A100E476E4850456E5E
:105D600038EC26F0110E476E4950456E38EC26F09F
:105D700012004AAE1200010E355CD8B0C4EF2EF00E
:105D80001A0E366EEAEF2EF00F0E355CD8B0CDEF5E
:105D90002EF0140E366EEAEF2EF01E0E355CD8B0E3
:105DA000D6EF2EF00C0E366EEAEF2EF02D0E355C8F
:105DB000D8B0DFEF2EF0060E366EEAEF2EF03C0E76
:105DC000355CD8B0E8EF2EF0030E366EEAEF2EF019
:105DD000010E366E51A2F0EF2EF051B4FFEF2EF00F
:105DE0003650396E0E0E485CD8B4FFEF2EF04806E0
:105DF0003906000E395CD8A4F2EF2EF0356A51A2B4
:105E000005EF2FF051A414EF2FF03650396E0E0E1F
:105E1000495CD8B414EF2FF049063906000E395CFE
:105E2000D8A407EF2FF0356A100E476E4850456E24
:105E300038EC26F0110E476E4950456E38EC26F0CE
:105E40001200000E155CD8A42AEF2FF01BEC26F0F0
:105E5000010E156E356A1200010E155CD8A434EFE0
:105E60002FF01BEC26F0156A356A1200E7EC2CF0D7
:105E7000F6EC2FF0ABEC24F0400EB7EC24F0BE0EA5
:105E8000DFEC24F06AEC38F0000E07EC25F0000E91
:105E900007EC25F0AEEC3BF054EC33F03150336EB0
:105EA0003250346E3306000E285CD8A468EF2FF011
:105EB00037B064EF2FF0000E335ED8A464EF2FF0FC
:105EC000AEEC3BF06BEF2FF0B8EC3BF06BEF2FF04C
:105ED000AEEC3BF028062C2A120E2C5CD8A452EF14
:105EE0002FF02C6AAEEC24F0400EB7EC24F0BE0E7E
:105EF000DFEC24F03306000E285CD8A490EF2FF0DE
:105F000037B08CEF2FF0000E335ED8A48CEF2FF05B
:105F1000AEEC3BF093EF2FF0B8EC3BF093EF2FF0AB
:105F2000AEEC3BF028062C2A150E2C5CD8A47AEF98
:105F30002FF02C6AE7EC2CF0ABEC24F0400EB7EC21
:105F400024F0BF0EDFEC24F0CAEC38F0000E07ECB2
:105F500025F0000E07EC25F0AEEC3BF03406000E09
:105F6000275CD8A4C4EF2FF037B0C0EF2FF0000E9D
:105F7000345ED8A4C0EF2FF0AEEC3BF0C7EF2FF0AB
:105F8000B8EC3BF0C7EF2FF0AEEC3BF027062C2A25
:105F9000120E2C5CD8A4AEEF2FF02C6AAEEC24F0DD
:105FA000400EB7EC24F0BF0EDFEC24F03406000EF8
:105FB000275CD8A4ECEF2FF037B0E8EF2FF0000EFD
:105FC000345ED8A4E8EF2FF0AEEC3BF0EFEF2FF00B
:105FD000B8EC3BF0EFEF2FF0AEEC3BF027062C2AAD
:105FE000150E2C5CD8A4D6EF2FF02C6A010EC26ED1
:105FF000C294C282C2B2FAEF2FF0000EC26EC45039
:10600000246EC350236E6DEC2AF0010EC26EC28462
:10601000C282C2B209EF30F0C450266EC350256E62
:10602000000EC26EE7EC2CF019EC30F06DEC2AF0AB
:10603000120024B220EF30F0241E030E2416231E7B
:1060400024B050EF31F0030E235CD8B02CEF30F0C9
:10605000000E286E88EF31F0050E235CD8B035EFC6
:1060600030F0010E286E88EF31F0070E235CD8B0B7
:106070003EEF30F0020E286E88EF31F0080E235C00
:10608000D8B047EF30F0030E286E88EF31F0090EDC
:10609000235CD8B050EF30F0040E286E88EF31F05A
:1060A0000A0E235CD8B059EF30F0050E286E88EF49
:1060B00031F00B0E235CD8B062EF30F0060E286E84
:1060C00088EF31F00D0E235CD8B06BEF30F0070E87
:1060D000286E88EF31F00E0E235CD8B074EF30F0EC
:1060E000080E286E88EF31F0100E235CD8B07DEFDB
:1060F00030F0090E286E88EF31F0120E235CD8B014
:1061000086EF30F00A0E286E88EF31F0140E235C13
:10611000D8B08FEF30F00B0E286E88EF31F0170EED
:10612000235CD8B098EF30F00C0E286E88EF31F079
:10613000190E235CD8B0A1EF30F00D0E286E88EF59
:1061400031F01D0E235CD8B0AAEF30F00E0E286E91
:1061500088EF31F0200E235CD8B0B3EF30F00F0E93
:10616000286E88EF31F0240E235CD8B0BCEF30F0FD
:10617000100E286E88EF31F0290E235CD8B0C5EFE1
:1061800030F0110E286E88EF31F02E0E235CD8B05F
:10619000CEEF30F0120E286E88EF31F0330E235C14
:1061A000D8B0D7EF30F0130E286E88EF31F0390EEB
:1061B000235CD8B0E0EF30F0140E286E88EF31F099
:1061C000400E235CD8B0E9EF30F0150E286E88EF52
:1061D00031F0490E235CD8B0F2EF30F0160E286E85
:1061E00088EF31F0510E235CD8B0FBEF30F0170E82
:1061F000286E88EF31F05B0E235CD8B004EF31F0ED
:10620000180E286E88EF31F0660E235CD8B00DEFC3
:1062100031F0190E286E88EF31F0720E235CD8B081
:1062200016EF31F01A0E286E88EF31F0800E235CE5
:10623000D8B01FEF31F01B0E286E88EF31F0900EB2
:10624000235CD8B028EF31F01C0E286E88EF31F0B7
:10625000A10E235CD8B031EF31F01D0E286E88EF0F
:1062600031F0B50E235CD8B03AEF31F01E0E286E37
:1062700088EF31F0CB0E235CD8B043EF31F01F0E26
:10628000286E88EF31F0E40E235CD8B04CEF31F08B
:10629000200E286E88EF31F0210E286E88EF31F045
:1062A000000E235CD8A459EF31F0210E286E88EF40
:1062B00031F01F0E235CD8B062EF31F0220E286E51
:1062C00088EF31F0420E235CD8B06BEF31F0230E33
:1062D000286E88EF31F06A0E235CD8B074EF31F08D
:1062E000240E286E88EF31F0960E235CD8B07DEF37
:1062F00031F0250E286E88EF31F0C70E235CD8B040
:1063000086EF31F0260E286E88EF31F0270E286ECA
:106310006DEC2AF026B291EF31F0261E030E261600
:10632000251E26B0C1EF32F0030E255CD8B09DEFDC
:1063300031F0000E276EFBEF32F0050E255CD8B071
:10634000A6EF31F0010E276EFBEF32F0070E255C51
:10635000D8B0AFEF31F0020E276EFBEF32F0080E2F
:10636000255CD8B0B8EF31F0030E276EFBEF32F0AA
:10637000090E255CD8B0C1EF31F0040E276EFBEF9B
:1063800032F00A0E255CD8B0CAEF31F0050E276E48
:10639000FBEF32F00B0E255CD8B0D3EF31F0060ED8
:1063A000276EFBEF32F00D0E255CD8B0DCEF31F03C
:1063B000070E276EFBEF32F00E0E255CD8B0E5EF2E
:1063C00031F0080E276EFBEF32F0100E255CD8B0CE
:1063D000EEEF31F0090E276EFBEF32F0120E255C66
:1063E000D8B0F7EF31F00A0E276EFBEF32F0140E43
:1063F000255CD8B000EF32F00B0E276EFBEF32F0C9
:10640000170E255CD8B009EF32F00C0E276EFBEFAB
:1064100032F0190E255CD8B012EF32F00D0E276E57
:10642000FBEF32F01D0E255CD8B01BEF32F00E0EE4
:10643000276EFBEF32F0200E255CD8B024EF32F04F
:106440000F0E276EFBEF32F0240E255CD8B02DEF37
:1064500032F0100E276EFBEF32F0290E255CD8B01B
:1064600036EF32F0110E276EFBEF32F02E0E255C68
:10647000D8B03FEF32F0120E276EFBEF32F0330E42
:10648000255CD8B048EF32F0130E276EFBEF32F0E8
:10649000390E255CD8B051EF32F0140E276EFBEFA9
:1064A00032F0400E255CD8B05AEF32F0150E276E50
:1064B000FBEF32F0490E255CD8B063EF32F0160ED8
:1064C000276EFBEF32F0510E255CD8B06CEF32F046
:1064D000170E276EFBEF32F05B0E255CD8B075EF20
:1064E00032F0180E276EFBEF32F0660E255CD8B046
:1064F0007EEF32F0190E276EFBEF32F0720E255C44
:10650000D8B087EF32F01A0E276EFBEF32F0800E14
:10651000255CD8B090EF32F01B0E276EFBEF32F007
:10652000900E255CD8B099EF32F01C0E276EFBEF71
:1065300032F0A10E255CD8B0A2EF32F01D0E276E0E
:10654000FBEF32F0B50E255CD8B0ABEF32F01E0E8B
:10655000276EFBEF32F0CB0E255CD8B0B4EF32F0F3
:106560001F0E276EFBEF32F0E40E255CD8B0BDEFB6
:1065700032F0200E276EFBEF32F0210E276EFBEF7C
:1065800032F0000E255CD8A4CAEF32F0210E276E3F
:10659000FBEF32F01F0E255CD8B0D3EF32F0220EA5
:1065A000276EFBEF32F0420E255CD8B0DCEF32F004
:1065B000230E276EFBEF32F06A0E255CD8B0E5EFB4
:1065C00032F0240E276EFBEF32F0960E255CD8B029
:1065D000EEEF32F0250E276EFBEF32F0C70E255C92
:1065E000D8B0F7EF32F0260E276EFBEF32F0270E11
:1065F000276EFBEF32F02A50285CD8B024EF33F03E
:10660000000E2A5CD8B424EF33F02E2A000E415C31
:10661000D8A40EEF33F0030E17EF33F0010E415CF8
:10662000D8A416EF33F0040E17EF33F0060E2E5CED
:10663000D8A420EF33F02A062A50286E24EF33F036
:106640002A50286E25EF33F02E6A2950275CD8B0E7
:106650004FEF33F0000E295CD8B44FEF33F02D2A02
:10666000000E415CD8A438EF33F0030E41EF33F055
:10667000010E415CD8A440EF33F0040E41EF33F03B
:10668000060E2D5CD8A44AEF33F029062950276E58
:106690004EEF33F02950276E4FEF33F02D6A28501C
:1066A0002A6E2750296E120037B282EF33F0325033
:1066B000275CD8A061EF33F02750326E306A6CEF60
:1066C00033F0820E305CD8B469EF33F0302A6CEFCF
:1066D00033F0306A2750326E3150285CD8A076EF04
:1066E00033F02850316E2F6A81EF33F0820E2F5C29
:1066F000D8B47EEF33F02F2A81EF33F02F6A285081
:10670000316E12003250275CD8A08DEF33F0275045
:10671000326E306A1F92A9EF33F01FB298EF33F058
:10672000550E305CD8B498EF33F0302AA9EF33F02F
:10673000306A1F82000E325CD8B4A9EF33F0060E27
:10674000445CD8B4A7EF33F0442AA9EF33F0446A8D
:1067500032063150285CD8A0B4EF33F02850316EA7
:106760002F6A1F94D0EF33F01FB4BFEF33F0550EF4
:106770002F5CD8B4BFEF33F02F2AD0EF33F02F6A5D
:106780001F84000E315CD8B4D0EF33F0060E435CAA
:10679000D8B4CEEF33F0432AD0EF33F0436A31065A
:1067A0001200070E546EAEEC24F0400EB7EC24F04D
:1067B000BD0EDFEC24F054501D5CD8A4F7EF33F08D
:1067C00053AEEDEF33F0FF0E07EC25F09AEC35F009
:1067D000FF0E07EC25F00CEF34F0FF0E07EC25F070
:1067E0008AEC35F0FF0E07EC25F00CEF34F053AED9
:1067F00004EF34F0000E07EC25F0FAEC34F0000E54
:1068000007EC25F00CEF34F0000E07EC25F0EAEC75
:1068100034F0000E07EC25F0000E545CD8B415EFF0
:1068200034F054065346DBEF33F05346AEEC24F01D
:10683000530EB7EC24F0BE0EDFEC24F0080E1D5C06
:10684000D8A437EF34F0FF0E07EC25F09AEC3AF0BD
:10685000FF0E07EC25F0BAEC39F0FF0E07EC25F03F
:10686000AAEC3AF0FF0E07EC25F049EF34F0000EE9
:1068700007EC25F0DAEC38F0000E07EC25F00AEC16
:1068800038F0000E07EC25F0EAEC38F0000E07ECCB
:1068900025F012007C0E07EC25F0820E07EC25F0A7
:1068A000820E07EC25F0820E07EC25F07C0E07EC3B
:1068B00025F01200000E07EC25F0840E07EC25F001
:1068C000FE0E07EC25F0800E07EC25F0000E07EC1D
:1068D00025F01200E20E07EC25F0920E07EC25F0F1
:1068E000920E07EC25F0920E07EC25F08C0E07ECCB
:1068F00025F01200440E07EC25F0820E07EC25F07F
:10690000920E07EC25F0920E07EC25F06C0E07ECCA
:1069100025F01200300E07EC25F0280E07EC25F0CC
:10692000240E07EC25F0FE0E07EC25F0200E07ECF8
:1069300025F012004E0E07EC25F08A0E07EC25F02C
:106940008A0E07EC25F08A0E07EC25F0720E07EC94
:1069500025F012007C0E07EC25F0920E07EC25F0D6
:10696000920E07EC25F0920E07EC25F0640E07EC72
:1069700025F01200060E07EC25F0020E07EC25F0BC
:10698000C20E07EC25F0320E07EC25F00E0E07ECD8
:1069900025F012006C0E07EC25F0920E07EC25F0A6
:1069A000920E07EC25F0920E07EC25F06C0E07EC2A
:1069B00025F012004C0E07EC25F0920E07EC25F0A6
:1069C000920E07EC25F0920E07EC25F07C0E07ECFA
:1069D00025F012003C0E07EC25F0420E07EC25F0E6
:1069E000420E07EC25F0420E07EC25F03C0E07ECBA
:1069F00025F01200000E07EC25F0440E07EC25F000
:106A00007E0E07EC25F0400E07EC25F0000E07EC9B
:106A100025F01200720E07EC25F04A0E07EC25F067
:106A20004A0E07EC25F04A0E07EC25F0440E07EC61
:106A300025F01200220E07EC25F04A0E07EC25F097
:106A40004A0E07EC25F04A0E07EC25F0340E07EC51
:106A500025F01200300E07EC25F0280E07EC25F08B
:106A6000240E07EC25F07E0E07EC25F0200E07EC37
:106A700025F012002E0E07EC25F04A0E07EC25F04B
:106A80004A0E07EC25F04A0E07EC25F0320E07EC13
:106A900025F012003C0E07EC25F04A0E07EC25F01D
:106AA0004A0E07EC25F04A0E07EC25F0300E07ECF5
:106AB00025F01200060E07EC25F0020E07EC25F07B
:106AC000620E07EC25F0120E07EC25F00E0E07EC17
:106AD00025F01200340E07EC25F04A0E07EC25F0E5
:106AE0004A0E07EC25F04A0E07EC25F0340E07ECB1
:106AF00025F012000C0E07EC25F0520E07EC25F0E5
:106B0000520E07EC25F0520E07EC25F03C0E07EC78
:106B100025F01200C30E07EC25F0BD0E07EC25F0A2
:106B2000BD0E07EC25F0BD0E07EC25F0C30E07ECFB
:106B300025F01200FF0E07EC25F0BB0E07EC25F048
:106B4000810E07EC25F0BF0E07EC25F0FF0E07ECD9
:106B500025F012008D0E07EC25F0B50E07EC25F0A0
:106B6000B50E07EC25F0B50E07EC25F0BB0E07ECD3
:106B700025F01200DD0E07EC25F0B50E07EC25F030
:106B8000B50E07EC25F0B50E07EC25F0CB0E07ECA3
:106B900025F01200CF0E07EC25F0D70E07EC25F0FC
:106BA000DB0E07EC25F0810E07EC25F0DF0E07EC7D
:106BB00025F01200D10E07EC25F0B50E07EC25F0FC
:106BC000B50E07EC25F0B50E07EC25F0CD0E07EC61
:106BD00025F01200C30E07EC25F0B50E07EC25F0EA
:106BE000B50E07EC25F0B50E07EC25F0CF0E07EC3F
:106BF00025F01200F90E07EC25F0FD0E07EC25F04C
:106C00009D0E07EC25F0ED0E07EC25F0F10E07ECDC
:106C100025F01200CB0E07EC25F0B50E07EC25F0A1
:106C2000B50E07EC25F0B50E07EC25F0CB0E07EC02
:106C300025F01200F30E07EC25F0AD0E07EC25F061
:106C4000AD0E07EC25F0AD0E07EC25F0C30E07ECFA
:106C500025F01200F80E07EC25F0240E07EC25F0C5
:106C6000220E07EC25F0240E07EC25F0F80E07ECB9
:106C700025F01200FE0E07EC25F0920E07EC25F031
:106C8000920E07EC25F0920E07EC25F06C0E07EC47
:106C900025F012007C0E07EC25F0820E07EC25F0A3
:106CA000820E07EC25F0820E07EC25F0440E07EC6F
:106CB00025F01200FE0E07EC25F0820E07EC25F001
:106CC000820E07EC25F0820E07EC25F07C0E07EC17
:106CD00025F01200FE0E07EC25F0920E07EC25F0D1
:106CE000920E07EC25F0920E07EC25F0820E07ECD1
:106CF00025F01200FE0E07EC25F0120E07EC25F031
:106D0000120E07EC25F0120E07EC25F0020E07EC30
:106D100025F012007C0E07EC25F0820E07EC25F022
:106D2000820E07EC25F0920E07EC25F0740E07ECAE
:106D300025F01200FE0E07EC25F0100E07EC25F0F2
:106D4000100E07EC25F0100E07EC25F0FE0E07ECF8
:106D500025F01200000E07EC25F0820E07EC25F05E
:106D6000FE0E07EC25F0820E07EC25F0000E07EC76
:106D700025F01200600E07EC25F0800E07EC25F0E0
:106D8000800E07EC25F0800E07EC25F07E0E07EC58
:106D900025F01200FE0E07EC25F0100E07EC25F092
:106DA000280E07EC25F0440E07EC25F0820E07ECC8
:106DB00025F01200FE0E07EC25F0800E07EC25F002
:106DC000800E07EC25F0800E07EC25F0800E07EC16
:106DD00025F01200FE0E07EC25F0040E07EC25F05E
:106DE000080E07EC25F0040E07EC25F0FE0E07EC6C
:106DF00025F01200FE0E07EC25F0080E07EC25F03A
:106E0000100E07EC25F0200E07EC25F0FE0E07EC27
:106E100025F012007C0E07EC25F0820E07EC25F021
:106E2000820E07EC25F0820E07EC25F07C0E07ECB5
:106E300025F01200FE0E07EC25F0120E07EC25F0EF
:106E4000120E07EC25F0120E07EC25F00C0E07ECE5
:106E500025F012007C0E07EC25F0820E07EC25F0E1
:106E6000A20E07EC25F0420E07EC25F0BC0E07EC55
:106E700025F01200FE0E07EC25F0120E07EC25F0AF
:106E8000120E07EC25F0120E07EC25F0EC0E07ECC5
:106E900025F012004C0E07EC25F0920E07EC25F0C1
:106EA000920E07EC25F0920E07EC25F0640E07EC2D
:106EB00025F01200020E07EC25F0020E07EC25F07B
:106EC000FE0E07EC25F0020E07EC25F0020E07EC93
:106ED00025F012007E0E07EC25F0800E07EC25F061
:106EE000800E07EC25F0800E07EC25F07E0E07ECF7
:106EF00025F012000E0E07EC25F0300E07EC25F001
:106F0000C00E07EC25F0300E07EC25F00E0E07EC56
:106F100025F012001E0E07EC25F0E00E07EC25F020
:106F2000180E07EC25F0E00E07EC25F01E0E07EC1E
:106F300025F01200C60E07EC25F0280E07EC25F010
:106F4000100E07EC25F0280E07EC25F0C60E07EC16
:106F500025F012000E0E07EC25F0100E07EC25F0C0
:106F6000E00E07EC25F0100E07EC25F00E0E07ECF6
:106F700025F01200C20E07EC25F0A20E07EC25F05A
:106F8000920E07EC25F08A0E07EC25F0860E07EC32
:106F900025F01200780E07EC25F0140E07EC25F012
:106FA000120E07EC25F0140E07EC25F0780E07EC16
:106FB00025F012007E0E07EC25F04A0E07EC25F0B6
:106FC0004A0E07EC25F04A0E07EC25F0340E07ECCC
:106FD00025F012003C0E07EC25F0420E07EC25F0E0
:106FE000420E07EC25F0420E07EC25F0240E07ECCC
:106FF00025F012007E0E07EC25F0420E07EC25F07E
:10700000420E07EC25F0420E07EC25F03C0E07EC93
:1070100025F012007E0E07EC25F04A0E07EC25F055
:107020004A0E07EC25F04A0E07EC25F0420E07EC5D
:1070300025F012007E0E07EC25F00A0E07EC25F075
:107040000A0E07EC25F00A0E07EC25F0020E07ECFD
:1070500025F012003C0E07EC25F0420E07EC25F05F
:10706000420E07EC25F0520E07EC25F0340E07EC2B
:1070700025F012007E0E07EC25F0080E07EC25F037
:10708000080E07EC25F0080E07EC25F07E0E07EC45
:1070900025F01200000E07EC25F0420E07EC25F05B
:1070A0007E0E07EC25F0420E07EC25F0000E07ECF3
:1070B00025F012007E0E07EC25F0100E07EC25F0EF
:1070C000080E07EC25F0140E07EC25F0620E07EC15
:1070D00025F012007E0E07EC25F0400E07EC25F09F
:1070E000400E07EC25F0400E07EC25F0400E07ECB3
:1070F00025F012007E0E07EC25F0040E07EC25F0BB
:10710000080E07EC25F0040E07EC25F07E0E07ECC8
:1071100025F012007E0E07EC25F0040E07EC25F09A
:10712000180E07EC25F0200E07EC25F07E0E07EC7C
:1071300025F012003C0E07EC25F0420E07EC25F07E
:10714000420E07EC25F0420E07EC25F03C0E07EC52
:1071500025F012007E0E07EC25F0120E07EC25F04C
:10716000120E07EC25F0120E07EC25F00C0E07ECC2
:1071700025F012003C0E07EC25F0420E07EC25F03E
:10718000520E07EC25F0220E07EC25F05C0E07EC02
:1071900025F012007E0E07EC25F0120E07EC25F00C
:1071A000120E07EC25F0120E07EC25F06C0E07EC22
:1071B00025F01200440E07EC25F04A0E07EC25F0EE
:1071C0004A0E07EC25F04A0E07EC25F0320E07ECCC
:1071D00025F01200020E07EC25F0020E07EC25F058
:1071E0007E0E07EC25F0020E07EC25F0020E07ECF0
:1071F00025F012003E0E07EC25F0400E07EC25F0BE
:10720000400E07EC25F0400E07EC25F03E0E07EC93
:1072100025F01200060E07EC25F0180E07EC25F0FD
:10722000600E07EC25F0180E07EC25F0060E07ECB3
:1072300025F012007E0E07EC25F0200E07EC25F05D
:10724000100E07EC25F0200E07EC25F07E0E07EC63
:1072500025F01200460E07EC25F0280E07EC25F06D
:10726000100E07EC25F0280E07EC25F0460E07EC73
:1072700025F01200060E07EC25F0080E07EC25F0AD
:10728000700E07EC25F0080E07EC25F0060E07EC53
:1072900025F01200440E07EC25F0640E07EC25F0F3
:1072A000540E07EC25F04C0E07EC25F0440E07ECCD
:1072B00025F01200300E07EC25F0480E07EC25F003
:1072C000480E07EC25F0480E07EC25F07E0E07EC83
:1072D00025F01200CF0E07EC25F0B70E07EC25F0D5
:1072E000B70E07EC25F0B70E07EC25F0810E07EC82
:1072F00025F01200870E07EC25F0EB0E07EC25F0C9
:10730000ED0E07EC25F0EB0E07EC25F0870E07ECF1
:1073100025F01200810E07EC25F0B50E07EC25F0E4
:10732000B50E07EC25F0B50E07EC25F0CB0E07ECFB
:1073300025F01200C30E07EC25F0BD0E07EC25F07A
:10734000BD0E07EC25F0BD0E07EC25F0DB0E07ECBB
:1073500025F01200810E07EC25F0BD0E07EC25F09C
:10736000BD0E07EC25F0BD0E07EC25F0C30E07ECB3
:1073700025F01200810E07EC25F0B50E07EC25F084
:10738000B50E07EC25F0B50E07EC25F0BD0E07ECA9
:1073900025F01200810E07EC25F0F50E07EC25F024
:1073A000F50E07EC25F0F50E07EC25F0FD0E07ECC9
:1073B00025F01200C30E07EC25F0BD0E07EC25F0FA
:1073C000BD0E07EC25F0AD0E07EC25F0CB0E07EC5B
:1073D00025F01200810E07EC25F0F70E07EC25F0E2
:1073E000F70E07EC25F0F70E07EC25F0810E07EC01
:1073F00025F01200FF0E07EC25F0BD0E07EC25F07E
:10740000810E07EC25F0BD0E07EC25F0FF0E07EC12
:1074100025F01200CF0E07EC25F0BF0E07EC25F08B
:10742000BF0E07EC25F0BF0E07EC25F0C10E07ECF0
:1074300025F01200810E07EC25F0EF0E07EC25F089
:10744000F70E07EC25F0EB0E07EC25F09D0E07EC90
:1074500025F01200810E07EC25F0BF0E07EC25F099
:10746000BF0E07EC25F0BF0E07EC25F0BF0E07ECB2
:1074700025F01200810E07EC25F0FB0E07EC25F03D
:10748000F70E07EC25F0FB0E07EC25F0810E07EC5C
:1074900025F01200810E07EC25F0FB0E07EC25F01D
:1074A000E70E07EC25F0DF0E07EC25F0810E07EC68
:1074B00025F01200C30E07EC25F0BD0E07EC25F0F9
:1074C000BD0E07EC25F0BD0E07EC25F0C30E07EC52
:1074D00025F01200810E07EC25F0ED0E07EC25F0EB
:1074E000ED0E07EC25F0ED0E07EC25F0F30E07ECA2
:1074F00025F01200C30E07EC25F0BD0E07EC25F0B9
:10750000AD0E07EC25F0DD0E07EC25F0A30E07EC21
:1075100025F01200810E07EC25F0ED0E07EC25F0AA
:10752000ED0E07EC25F0ED0E07EC25F0930E07ECC1
:1075300025F01200BB0E07EC25F0B50E07EC25F088
:10754000B50E07EC25F0B50E07EC25F0CD0E07ECD7
:1075500025F01200FD0E07EC25F0FD0E07EC25F0DE
:10756000810E07EC25F0FD0E07EC25F0FD0E07EC73
:1075700025F01200C10E07EC25F0BF0E07EC25F038
:10758000BF0E07EC25F0BF0E07EC25F0C10E07EC8F
:1075900025F01200F90E07EC25F0E70E07EC25F0B8
:1075A0009F0E07EC25F0E70E07EC25F0F90E07EC2F
:1075B00025F01200810E07EC25F0DF0E07EC25F018
:1075C000EF0E07EC25F0DF0E07EC25F0810E07EC3F
:1075D00025F01200B90E07EC25F0D70E07EC25F0C8
:1075E000EF0E07EC25F0D70E07EC25F0B90E07ECEF
:1075F00025F01200F90E07EC25F0F70E07EC25F048
:107600008F0E07EC25F0F70E07EC25F0F90E07ECCE
:1076100025F012009D0E07EC25F0AD0E07EC25F0CD
:10762000B50E07EC25F0B90E07EC25F0BD0E07EC02
:1076300025F01200000E07EC25F0000E07EC25F0F7
:10764000040E07EC25F00A0E07EC25F0040E07ECFB
:1076500025F01200000E07EC25F0000E07EC25F0D7
:10766000000E07EC25F0000E07EC25F0000E07ECED
:1076700025F01200FF0E07EC25F0FF0E07EC25F0B9
:10768000FF0E07EC25F0FF0E07EC25F0FF0E07ECD0
:1076900025F01200280E07EC25F01200280E07EC4A
:1076A00025F0280E07EC25F0280E07EC25F0280E13
:1076B00007EC25F0280E07EC25F01200100E07EC61
:1076C00025F0100E07EC25F07C0E07EC25F0100ECF
:1076D00007EC25F0100E07EC25F01200100E07EC59
:1076E00025F0100E07EC25F0100E07EC25F0100E1B
:1076F00007EC25F0100E07EC25F01200EF0E07EC5A
:1077000025F0EF0E07EC25F0EF0E07EC25F0EF0E5D
:1077100007EC25F0EF0E07EC25F01200400E07EC09
:1077200025F0200E07EC25F0100E07EC25F0080ED2
:1077300007EC25F0040E07EC25F01200BF0E07EC55
:1077400025F0DF0E07EC25F0EF0E07EC25F0F70E25
:1077500007EC25F0FB0E07EC25F012007E0E07EC7F
:1077600025F07E0E07EC25F0000E07EC25F0120048
:10777000000E07EC25F0000E07EC25F0000E07ECDC
:1077800025F01200CAEC37F0000E07EC25F0FAECF9
:1077900037F0000E07EC25F0FAEC37F0000E07EC9E
:1077A00025F0CAEC38F0000E07EC25F00AEC38F0B2
:1077B000000E07EC25F0DAEC38F0000E07EC25F0AF
:1077C000DAEC38F02AEC3BF01200000EAA6E000E44
:1077D000A96E4850A86EA69EA69CA684550EA76EBC
:1077E000AA0EA76EA682A6B2F3EF3BF0A6941200F3
:1077F000000EAA6E010EA96E4950A86EA69EA69C08
:10780000A684550EA76EAA0EA76EA682A6B206EF94
:107810003CF0A6941200000EAA6E020EA96E4A5009
:10782000A86EA890A69EA69CA684550EA76EAA0E2A
:10783000A76EA682A6B21AEF3CF0A6941200000E24
:10784000AA6E030EA96E4B50A86EA69EA69CA68497
:10785000550EA76EAA0EA76EA682A6B22DEF3CF01B
:10786000A6941200000EAA6E040EA96E4C50A86ECB
:10787000A69EA69CA684550EA76EAA0EA76EA682EB
:10788000A6B240EF3CF0A6941200000EAA6E050EC0
:10789000A96E4D50A86EA69EA69CA684550EA76EF6
:1078A000AA0EA76EA682A6B253EF3CF0A6941200D1
:1078B000000EAA6E060EA96E5150A86EA69EA69C3A
:1078C000A684550EA76EAA0EA76EA682A6B266EF74
:1078D0003CF0A6941200000EAA6E070EA96E375057
:1078E000A86EA69EA69CA684550EA76EAA0EA76E8D
:1078F000A682A6B279EF3CF0A6941200000EAA6E02
:10790000080EA96E4150A86EA69EA69CA684550E90
:10791000A76EAA0EA76EA682A6B28CEF3CF0A69424
:02792000120053
:020000040030CA
:03000100381800AC
:02000500358044
:060008000FC00FE00F40E5
:0200000400F00A
:0A000000FFFFA00102000000010054
:00000001FF
